:020000040800F2
:1000000000200020514300084543000847430008F2
:1000100000000000000000000000000000000000E0
:10002000000000000000000000000000494300083C
:1000300000000000000000004B4300084D43000892
:10004000A143000800000000A1430008A1430008EC
:10005000A1430008A1430008A1430008A1430008F0
:1000600000000000A1430008A1430008A1430008CC
:10007000A1430008A1430008A143000800000000BC
:10008000A14300080000000000000000A143000898
:1000900000000000A1430008A1430008A14300089C
:1000A000A1430008A1430008A1430008A1430008A0
:0800B000A1430008000000005C
:1000B80010B5064C2378002B07D1054B002B02D036
:1000C800044800E000BF0123237010BDB0000020E9
:1000D800000000002C590008044B10B5002B03D079
:1000E8000349044800E000BF10BDC04600000000FE
:1000F800B40000202C5900080023C25C0133002AF8
:10010800FBD1581E7047000002B4714649084900E7
:10011800095649008E4402BC7047C0460022430875
:100128008B4274D303098B425FD3030A8B4244D3B7
:10013800030B8B4228D3030C8B420DD3FF220902F9
:1001480012BA030C8B4202D31212090265D0030BB8
:100158008B4219D300E0090AC30B8B4201D3CB03AE
:10016800C01A5241830B8B4201D38B03C01A5241F0
:10017800430B8B4201D34B03C01A5241030B8B42F2
:1001880001D30B03C01A5241C30A8B4201D3CB02DD
:10019800C01A5241830A8B4201D38B02C01A5241C2
:1001A800430A8B4201D34B02C01A5241030A8B42C5
:1001B80001D30B02C01A5241CDD2C3098B4201D3DD
:1001C800CB01C01A524183098B4201D38B01C01A5B
:1001D800524143098B4201D34B01C01A52410309D2
:1001E8008B4201D30B01C01A5241C3088B4201D381
:1001F800CB00C01A524183088B4201D38B00C01A2E
:10020800524143088B4201D34B00C01A5241411A54
:1002180000D20146524110467047FFE701B5002061
:1002280000F0F0F802BDC0460029F7D076E7704725
:1002380003460B437FD4002243088B4274D303093F
:100248008B425FD3030A8B4244D3030B8B4228D3E0
:10025800030C8B420DD3FF22090212BA030C8B4206
:1002680002D31212090265D0030B8B4219D300E0A6
:10027800090AC30B8B4201D3CB03C01A5241830B2B
:100288008B4201D38B03C01A5241430B8B4201D3DB
:100298004B03C01A5241030B8B4201D30B03C01A04
:1002A8005241C30A8B4201D3CB02C01A5241830A7E
:1002B8008B4201D38B02C01A5241430A8B4201D3AD
:1002C8004B02C01A5241030A8B4201D30B02C01AD7
:1002D8005241CDD2C3098B4201D3CB01C01A52413E
:1002E80083098B4201D38B01C01A524143098B42C7
:1002F80001D34B01C01A524103098B4201D30B01B0
:10030800C01A5241C3088B4201D3CB00C01A5241D4
:1003180083088B4201D38B00C01A524143088B4299
:1003280001D34B00C01A5241411A00D20146524132
:10033800104670475DE0CA0F00D04942031000D351
:100348004042534000229C4603098B422DD3030AA6
:100358008B4212D3FC22890112BA030A8B420CD3B6
:10036800890192118B4208D3890192118B4204D3DF
:1003780089013AD0921100E08909C3098B4201D35F
:10038800CB01C01A524183098B4201D38B01C01A99
:10039800524143098B4201D34B01C01A5241030910
:1003A8008B4201D30B01C01A5241C3088B4201D3BF
:1003B800CB00C01A524183088B4201D38B00C01A6C
:1003C8005241D9D243088B4201D34B00C01A524143
:1003D800411A00D20146634652415B10104601D3D0
:1003E8004042002B00D54942704763465B1000D35A
:1003F800404201B5002000F005F802BD0029F8D000
:1004080016E770477047C0468446100062468C461F
:100418001900634600E0C0461FB500F00DFF002834
:1004280001D40021C8421FBD10B500F05DFE404256
:10043800013010BD10B500F0FFFE002801DB0020E0
:1004480010BD012010BDC04610B500F0F5FE002813
:1004580001DD002010BD012010BDC04610B500F020
:1004680085FE002801DC002010BD012010BDC0461B
:1004780010B500F07BFE002801DA002010BD012035
:1004880010BDC046F0B54F464646D6460D0004009E
:10049800C0B51F0011002803620F400A10437A00FC
:1004A800520DE3003C039146640AFA0F4F0F6E00A9
:1004B80027439246B846760DED0FC900954200D104
:1004C80099E04C46341BA446002C00DC7CE04A46EC
:1004D800002A00D1B8E0C54A964200D11CE180222A
:1004E8003C0012041443A0466246382A00DD61E14C
:1004F8001F2A00DDCCE164462022121B44469440AA
:100508000F00A14664469140E7404C464A1E91417F
:100518003C43424621436446E240801A5C1AA342A7
:100528009B415F42C71B3B0200D4D0E07F027F0A99
:10053800002F00D1FFE0380001F08AFD01000839E2
:10054800202322005B1A8F40DA408C401743B142C7
:1005580000DAFFE0891B4B1C1F2B00DDA8E02022DE
:100568003900D21A200094409140D840621E94412C
:10057800DF40002601430C43630709D00F232340C3
:10058800042B05D0231DA342A44164423F191C003B
:100598003B0200D49EE0954B01369E4200D1B7E065
:1005A800934AE40817407B0771057F0223433F0BFA
:1005B8004A0D12053A43ED072A4318001100E0BC22
:1005C800BA46B146A846F0BD002C4BD04C46A41BF9
:1005D800A446002E00D023E104001C4300D1AFE163
:1005E8006246541E012A00D115E2804DAC4500D167
:1005F800C8E1A4461BE14A46B21A9446002A00DC28
:10060800ACE04A46002A43D0784A964200D1AFE18E
:1006180080223C0012041443A0466246382A67DC54
:100628001F2A00DC5FE14746203AD7406246202A6D
:1006380005D064464022121B4446944021434A1E7A
:1006480091410C003C4357E03A000A4300D105E1D0
:100658002200013A012C00D182E1644CA4455BD010
:10066800944641E7634C771C274200D0C4E004005D
:100678001C43002E00D069E1002C00D1BFE14446A4
:100688000C4300D0D0E14207DB081343C00829E03F
:100698003A000A4300D170E162466446013A012CEF
:1006A80000D1E0E0514CA44500D161E19446B4E7A3
:1006B8003A001F39CA401100202B03D04022D31A18
:1006C8009F403C43631E9C41002700260C43630760
:1006D80000D053E7B446E4087B072343F808434AAD
:1006E80094451DD06246070352053F0B520D60E743
:1006F80044460C43621E9441E4189C429B415F426D
:100708003F183B02E3D5394B01369E4200D0B5E095
:100718003200002700234CE74207DB081343C008D8
:100728001A00024300D1E1E180273F0307433F035A
:100738002E4A3F0B3DE7200001F08AFC01001831EA
:100748001F2900DCFCE60838844027000024B14259
:1007580000DBFFE6264A761A17400DE7002A2FD05D
:100768004A46921B9446002E00D1ADE01F4A91459F
:1007780000D10FE18022120410436246382A00DDBE
:100788000FE11F2A00DD80E1644620221E00121BB3
:100798006746040093409440FE405A1E9341F84037
:1007A80034431C43804464188C42BF417F424E4608
:1007B8004744A6E742460A4311004A1E9141ADE666
:1007C8000C4C721C224200D0A1E002001A43002EF9
:1007D80000D0FAE0002A00D145E13A000A4300D0EF
:1007E80046E14207DB081343C0087BE7FF07000028
:1007F800FFFF7FFFFE07000047465C1AC21BA342AB
:10080800BF417F42B94617004A46BF1A3A0200D58F
:100818008DE023003B4300D08AE60020002561E7F5
:10082800B44CA14500D1ADE08024240420436446A3
:10083800382C3DDC62461F2C00DDB7E020251E0069
:100848002D1B0400AB40AC40D640D04042465D1E54
:10085800AB413443121A904623432CE04207DB088D
:100868001343C0083BE75C189C429B4140445B42F1
:10087800C71801263B0200D429E702269E4A6308CE
:100888001740012214401C43FB071C437F0873E6F2
:100898004446203AD4406246202A05D06746402282
:1008A800D21B4746974039434A1E9141214335E6BA
:1008B8000343581E8341CC1AA142BF4143467F429D
:1008C80055464E46DF1B2EE602001A4300D1BDE016
:1008D80062466446013A012C00D1E5E0854CA44506
:1008E80058D0944649E764462022121B4446944057
:1008F8000F00A14664469140E7404C464A1E91418C
:100908003C4342460C436146CA408018F4E6794CA1
:10091800A24200D1FDE6591899429B4140445F42EA
:10092800C719FC07490816000C437F08CFE6CC1A04
:10093800A142BF4143467F42181A5546C71BF7E5F7
:10094800C9087B0755460B43F808C8E6002C00D0B9
:1009580081E043460B4315D1802000250003E3E6E0
:100968005C1AA3429B41C71B5B420126FF1ADAE5CA
:100978004207DB081343C008D2E64207DB081343EB
:10098800C008ACE643464246C9085B0755460B43D8
:10099800D008C5E6434642465B07C9080B43D00862
:1009A800BEE603431C00631E9C41FCE60200203C9B
:1009B800E24014006246202A03D04025AD1AA84020
:1009C8000343581E8341234375E7002AE2D03A00C7
:1009D8000A43CDD04207DB0813438022C008120324
:1009E800104206D0FC08144203D12000CB087A0735
:1009F80013435A0FDB005207DB08134390E64346C4
:100A08000B4300D109E743464246C9085B075546F0
:100A18000B43D00866E6CC1AA14289413F1A4942E5
:100A2800554601267F1A7EE542465C1A871AA3427C
:100A380092415242BF1A3A023DD5CC1AA14289418D
:100A4800434649421F1A55467F1A95E57B07C90850
:100A58000B43F80843E64446DB080C4330D1420711
:100A68001343C0085CE67B07C9080B43F80839E65E
:100A78005C189C429B4140445B42C7183B0200D42F
:100A880025E61D4B01261F4021E60400203AD440EC
:100A98006246202A04D040226646921B90400343B7
:100AA8005A1E93411C437EE65C188C42894140449F
:100AB80049424718DDE623003B4300D1ADE606E690
:100AC800440723438024C0082403204208D0424618
:100AD800D608264204D155463000CB0851070B43AF
:100AE8005A0FDB00DB085207134319E60023014ABB
:100AF8001F005EE5FF070000FFFF7FFFF0B55746C8
:100B08004E464546DE46E0B5814605000C034800E2
:100B180092461F0085B0240B400DCE0F002800D14F
:100B280056E1D44B984200D172E16B0FE4001C43AC
:100B380080231B0423439846CF4BED009B4600239C
:100B48009946834400933C037B005046240B5B0D7D
:100B5800FF0F002B00D11FE1C64A934200D162E18A
:100B6800C549420F8C46E400594614438022634429
:100B78001204CB1A14439B46C200002033007B406A
:100B88009A464B460F2B27D8BC499B00CB589F460B
:100B9800B246009B022B16D0032B00D18EE2012B0C
:100BA80000D0D9E000230024002552461B0523432A
:100BB800D20713432800190005B0F0BCBB46B24663
:100BC800A946A046F0BD00240025AA4BEDE7BA4689
:100BD800A04615000090DCE7444500D2C7E100D1EB
:100BE800C2E101235B429C462E0040460025E344B7
:100BF8002302140E1C431B0C994623041F0C1202DB
:100C0800494600920197FFF70FFB02007A430B0455
:100C1800310C804619438A4207D901235B429C461E
:100C28000919E0448C4200D807E2881A4946FFF7C0
:100C3800FBFA09048C4631046646019A090C4243C2
:100C4800030031438A4204D90919013B8C4200D878
:100C5800EDE1881A424612041A4390464146009B29
:100C68000E041B0C1F000293009B360C1B04190C6E
:100C78000B007343120C7E43039151437A431F0CBC
:100C8800BC4676186644B14203D9802149028C4695
:100C98006244310C8A1831041E04360C8E199042B5
:100CA80002D312D1B54210D24346591E009B9C462E
:100CB80065441F009D429B415B421B19C01884423A
:100CC80000D2A0E100D19BE18846AE1BB542AD4100
:100CD800801A6D42401B844200D1D5E14946FFF796
:100CE800A3FA019A0B044243310C050019438A42C6
:100CF80000D96CE1881A4946FFF796FA019A36043A
:100D080042430904360C03000E43B24200D953E1B2
:100D18000398B61A02002D041D43029F2B041B0CD6
:100D28005A437B439C46290C4843130C8444634430
:100D38007943984203D98020400284466144180CC4
:100D480012041B04120C41189B188E4200D2FFE0BB
:100D580000D1FAE001231D43494A5A44002A00DC25
:100D6800AAE06B0700D03DE1ED084346DB0106D55C
:100D78004246444B1A4090468022D2005A44424B85
:100D88009A4200DD1FE743465B071D434346520571
:100D98005C02240B530D08E75246224300D17BE046
:100DA800002C00D1FAE0200001F052F902000B3AC1
:100DB8001D2301009B1A52460839DA408C4014431F
:100DC80052468A40314B58449B4683440020D5E61E
:100DD8004B462343984644D0002C00D1CEE0200057
:100DE80001F036F9010002000B391D235B1A494650
:100DF8001000D940083884400B004D4623439846DC
:100E080085402348831A9B460023994600939AE617
:100E18004B46234398461DD108239946063B002597
:100E2800834600938FE65246224309D1022349465E
:100E38001943184B89469C4600240220E3449DE64A
:100E480003234A461A43134B91469C4652460320B5
:100E5800E34493E60C239946093BA0468346009356
:100E680071E60423994600239B460133002500932D
:100E780069E6C046FF07000001FCFFFF485900086B
:100E8800FF030000FFFFFFFEFE070000F303000062
:100E98000DFCFFFF01F8FFFF49460123194389466E
:100EA800002401206AE6002380249A4600258A4B04
:100EB80024037AE601256D4201239B1A382B00DDB5
:100EC80070E61F2B00DCBFE01F2149428A1A414609
:100ED800D1400A00202B04D04146804B5B44994006
:100EE8000D436B1E9D4107232A431D000024154016
:100EF800134200D1D4E00F2100231140042900D16E
:100F0800CBE0111D9142924152429B180A001902EE
:100F180000D4C2E001230024002546E68023414690
:100F28001B03194208D01C4206D11C432403BA46AD
:100F38001500694B240B38E68024434624031C43E0
:100F48002403B246644B240B2FE6002B00D103E7A1
:100F5800A619681EA64200D28DE08E4200D2A3E0F8
:100F680000D1B3E00500F5E6AA4200D939E64346C8
:100F7800DE0758086B081E43ED0739E6484601F0BE
:100F880067F801000200153120321C2900DC2CE72B
:100F98004B46083883400025984632E701F058F858
:100FA80003001A00153220301C2A00DC00E75446E2
:100FB800083B00229C4005E73619013BB44200D9A2
:100FC800A6E6B24200D8A3E6831E3619A0E60919A0
:100FD800013D8C4200D98DE68A4200D88AE6851EFA
:100FE800091987E60F232B40042B00D1BCE6052303
:100FF8005B42AB429B4104355B42ED089844B4E642
:10100800AF4200D960E6824204D800D05CE6AE4226
:1010180000D859E602235B429C46009BE0449C466C
:1010280065449D429B415B421B19C0184DE68A42AC
:1010380000D80EE6831E09190BE68A4200D8F4E5AB
:10104800831E98460919F0E52549280059448D4022
:1010580042468A40691E8D414146D840D9400243E4
:101068002A430B00510700D151E70F2111400429F1
:1010780000D046E74BE705008E4200D06AE6009AAA
:10108800934200D066E667E6164A5A44002A00DC16
:1010980010E701230025984467E65D075B021C0BF7
:1010A800D2080023154380E50098023D42008242A1
:1010B800BF417F423C1936190092DDE78024434640
:1010C80024031C432403044B240B6EE5009A9A4224
:1010D800EAD30500D3E7C046FF0700003E0400003E
:1010E8001E040000FF030000F0B54E464546DE46EC
:1010F80057469046E0B517001A03120B05008446C0
:1011080019480E034C0091465A00DB0F9B46360BDC
:10111800640DC90F520D844219D0824210D00120AB
:1011280094420ED14E450CD10120C44509D15945F0
:1011380017D0002C05D130002843431E984100E009
:101148000120F0BCBB46B246A946A046F0BD33001C
:1011580001202B43F5D1A242F3D14B463B43F0D1BA
:10116800E2E70020EDE7C046FF070000F0B547467C
:10117800CE460400180016001B031B0B2D4D4A0019
:10118800994680B543000F03A446B0463F0B520D65
:10119800C90F5B0DC00FAA4221D0AB4213D0002A61
:1011A80022D13C43002B02D14D462E4322D0002CA5
:1011B80010D0814222D00220013908400138C0BC39
:1011C800B946B046F0BD4D462E4329D1002AF0D18C
:1011D8003C43EED10028F2D101204042EFE73D0028
:1011E80025431DD19342EED0002BE2D14C46264335
:1011F800DFD1E0E70020002CE1D0DCE79A420ADCEE
:10120800E8DB4F45D7D80ED000204F45D7D200296C
:10121800E2D00800D3E74342584140000138CEE706
:1012280002204042CBE7C445C5D80020C445C6D2F9
:10123800EDE7C046FF070000F0B54746CE4604007C
:10124800180016001B031B0B2C4D4A00994680B54D
:1012580043000F03A446B0463F0B520DC90F5B0D68
:10126800C00FAA420DD0AB4210D0002A27D13C4370
:10127800002B11D14D462E430ED10020002C15D045
:101288000EE03D00254310D1934218D14D462E4320
:101298000BD1002A02D13C43002C0BD0814214D040
:1012A800022001390840013800E00220C0BCB946DC
:1012B800B046F0BD0028F9D101204042F6E7002BE6
:1012C800ECD14C462643E9D1EAE79A4204DD434291
:1012D800584140000138E9E79A42EBDB4F45DFD837
:1012E80006D000204F45E1D20029E5D00800DDE70F
:1012F800C445D5D80020C445D8D2F5E7FF0700007B
:10130800F0B557464E464546DE46E0B598460C03CE
:101318004B000600924687B0240B5B0DCF0F002BC5
:1013280000D15CE1D94A934200D175E1420FE40053
:101338001443802212041443D54AC50094466344DA
:101348000093002399469B46434642461E03D20F0C
:101358005B0050469046360B5B0D00D120E1CB4A2E
:10136800934200D162E1CA49420F8C460099634416
:10137800F6008C46164380229C44120463461643AA
:10138800C200002000930099434601318C4649462B
:101398007B4001930F2926D8BE4B890059588F46A8
:1013A800434601933400150083465B46022B16D052
:1013B800032B00D103E2012B00D0CDE00022002452
:1013C8000025019B12052243DB071A432800110060
:1013D80007B0F0BCBB46B246A946A046F0BD002403
:1013E8000025AA4AEDE7280C2D042D0C2B00110C22
:1013F8001204120C5343984613002F004343994696
:101408004F434F44BB4647460B003F0CBA46434345
:10141800DA440293D14504D980277F02B9464B4468
:10142800029353461B0C9B4653461F0443461B041A
:101438001B0C98463B0043440493330C3604360C8B
:101448009846330043439946434643432F009A4600
:10145800434677435D43380C4D444519A94503D9A4
:1014680080235B029946CA443F04280C3F0C2D0494
:10147800ED19270C2404240C0300200050437A4360
:1014880091463A0053440593030C9A464A436143F4
:1014980049445144AB44894503D980235B029946AA
:1014A8004A4400040B0C000C090409182000994652
:1014B800434670435C437E435F43030C9846A4193C
:1014C80044444A440397A64204D980235B029846C1
:1014D800474403972304029E9A46059B5E44984618
:1014E800AE42AD4176188E4289410004000C50444A
:1014F80040446D424719B846934649428946C34419
:10150800D94498428041A845AD41934592418945C7
:1015180089416D4240422843240C524249420A43C1
:10152800039B00198018C7184B46DC0D049B7502F5
:101538001D436A1E95414B46F60D7F0235435A02FC
:101548003C431543FB0100D41CE101216A080D400E
:101558001543E207154364084F496144002900DC3C
:10156800B0E06B0709D00F222A40042A05D02A1DB3
:10157800AA42AD416D4264191500E30104D58021EA
:10158800464AC90014406144454A914200DD26E7B5
:101598006207ED08640249051543240B4A0D10E75C
:1015A8005246324300D17FE0002E00D1DCE030000B
:1015B80000F04EFD02000B3A1D2301009B1A524613
:1015C8000839DA408E40164352468A40009B354916
:1015D800181A03008C46634400200093D3E62500C4
:1015E80005434AD0002C00D1B0E0200000F030FDC7
:1015F800010002000B391D2310005B1A3100350071
:1016080008388440D94085400C432648831A009303
:10161800002399469B4697E60500254326D10822D4
:1016280000930223002491469B468DE65246009B78
:10163800324310D1154900268C466344494600932D
:1016480002231943894602209DE65B460197022B37
:1016580000D0ADE6C3E60D4A0320944663444A46EB
:10166800009303231A43914652468CE60C220093BA
:101678000323050091469B4666E60423994600230A
:101688000093013300249B465EE6C046FF07000036
:1016980001FCFFFF88590008FF030000FFFFFFFE61
:1016A800FE0700000DFCFFFF494601231943894648
:1016B8000026012067E6002380240025434A019381
:1016C80024037EE60120401A382800DD76E61F282C
:1016D8005BDD1F2223005242511ACB4019002028FB
:1016E80003D03B4A6244944025436A1E95412A0030
:1016F8000A4307210D000024154011425BD00F2139
:1017080000241140042953D0111D914292415242A4
:10171800A4180A0023024BD501220024002550E614
:1017280080231B031C4209D01E4207D133431C03EC
:1017380043461500240B254A019342E680221203F2
:1017480014432403214A240B01973AE600F080FC55
:1017580001000200153120321C2900DC4BE734005F
:1017680008380025844050E700F072FC03001A0096
:10177800153220301C2A00DC1EE75646083B0022A2
:101788009E4023E7009B9C46E6E6124922006144FE
:101798002E008D408A40C640691E8D4132432A433F
:1017A800C4405307B6D00F2111400429ACD1B1E78A
:1017B80065076402240BD2081543002201E6802243
:1017C800120314432403014A240BFAE5FF0700001F
:1017D8003E0400001E040000F8B557464E46454634
:1017E800DE46E0B51E0017004A000B03520D5B0AE7
:1017F8009046420F1A43CD0FCD4C3103C300944697
:1018080070007A0F490AFF009A46B946400DF60F54
:101818001143A04200D1B1E001225640B346B5427F
:1018280000D188E04246121A002A00DCAEE0002807
:1018380000D1C1E0BE48804500D151E180200004BC
:101848000143382A00DD7BE11F2A00DDEEE120207C
:101858003E00801A0C00D640D14087406246844042
:10186800521A781E8741944634432743DC1BA3420F
:101878009B4162465B42D31A99464B461B0200D4F1
:1018880018E14B465802430A99464B46002B00D1B3
:1018980037E1484600F0DCFB01000839202322002C
:1018A80048465B1ADA4088408C40434610438845D6
:1018B80000DD36E1C91A4B1C1F2B00DDEAE02022AF
:1018C8002600D21A01009440DE40D84000239140FF
:1018D800621E94418146984631430C43630709D000
:1018E8000F232340042B05D0231DA342A4416442A7
:1018F800A1441C004B461B0200D4DEE041468C4B41
:101908000131994200D1E7E04B468A48E408034098
:10191800180049055B07400223434A0D040B1205D2
:10192800ED0722432A4318001100F0BCBB46B2461B
:10193800A946A046F8BD4246121A002A52DD0028E0
:1019480000D19CE0A04500D1CAE0802000040143FA
:10195800382A00DD49E11F2A00DC97E110000E005B
:101968002038C640202A04D04020821A91400F43D4
:10197800B9464C46621E944134433AE10A003A4360
:1019880028D0B346B5422BD06B4A4244002A5DD0DA
:1019980042464446821A002C00D0F5E065461D43B5
:1019A80000D19CE1551E012A00D1FBE1604CA24206
:1019B80000D1BDE12A00F0E00800384300D1C3E0BF
:1019C800501E012A00D1A8E1594CA24200D187E05B
:1019D800020036E701225640B346B54200D021E75F
:1019E800554A4244002A00D1B5E042464446821A8C
:1019F800002C00D138E14E4EB04200D1DEE1802605
:101A0800644636043443A446382A00DD96E11F2A8A
:101A180000DD24E22026B41AA24664465646B440A5
:101A2800A1461C004E46D440264334005646B340D7
:101A38005E1EB3411C436346D340C918E419BC4237
:101A4800BF417F42B94680468944D8E040463B4C76
:101A58000130204200D0B4E04046002800D044E1E4
:101A68006046184300D190E10800384300D0AAE14D
:101A78006146DB0849070B436146CC0827E00800AC
:101A8800384361D0501E012A00D139E1A24227D043
:101A980002005DE702001F39CA401100202B03D065
:101AA8004022D31A98400443631E9C410023994660
:101AB80098460C43630700D012E74B464A46E408B1
:101AC8005B072343D408424619498A420ED02403AF
:101AD8005205240B520D22E70A00002400231EE7BA
:101AE800DB086246520713436246D4081A002243B1
:101AF80000D1FCE180221203144324030C4A240B76
:101B08000DE7200000F0A4FA010018311F2900DCBD
:101B1800C4E608388440434620000024884500DC99
:101B2800C8E6044A5B1A104098468146D6E6C04685
:101B3800FF070000FFFF7FFF01F8FFFFFE0700001F
:101B48000F437A1E974191E66146DB0849070B432C
:101B58006146CC08B8E74046D34C0130204200D05B
:101B6800A2E04046002800D001E16046184300D1B9
:101B78005EE10800384300D05FE16146DB084907B1
:101B88000B436146CC08A2E7C84DA84200D1CFE07C
:101B9800802564462D042C43A446382A56DC1F2A87
:101BA80000DDD1E020251E00AD1A6446AB40AC40F4
:101BB800D6405D1EAB41344323436446D440091BE1
:101BC80049E06046DC1B461AA342804140428146F8
:101BD80030004E46801B8146000276D44B46234394
:101BE80000D052E60024002571E739430C00621E3C
:101BF8009441E4189C429B415B42634499464B469E
:101C08001B0200D456E701239C46A84BE0449845A4
:101C180038D04B46A64801220340180063081440F8
:101C28001C43C3071C434308994657E610000E009F
:101C38002038C640202A04D04020821A91400F4301
:101C4800B9464F467A1E974137430FE662461A4314
:101C580013005A1E9341FC1AA742BF417F42CB1B77
:101C680099465D46804608E666461E4300D1BEE0BA
:101C7800561E012A00D109E18C4CA24200D119E17B
:101C88003200C1E642460024002348E620200C002A
:101C9800801A3E0087408440D640781E8741D14054
:101CA80034433C438C44A4E7804A904200D1E9E0A5
:101CB800DF199F429B4161445B42C918CC077F08EA
:101CC8004B08994680463C43F4E6FC1AA742BF41BC
:101CD80063467F42C91ACB1B99465D46D5E5FF0886
:101CE8004B075D463B43CC08EEE662461A4300D0FC
:101CF80082E00B003B431BD1802400252403F9E636
:101D0800DC199C429B41614489465B4299444B469D
:101D18001B0244D401239846CCE6DC1B6246A3424E
:101D28009B41511A5B42CB1A994601239846A4E578
:101D3800FF084B075D463B43CC08D7E662461A438B
:101D48001400631E9C4179E615006446203DEC4072
:101D5800A046202A05D040256446AA1A9440234369
:101D68009A465446631E9C414346234373E76246A2
:101D78001A4323D00A003A4300D0A0E06246DB08A9
:101D8800520713436246D408B0E60B003B4300D128
:101D980028E7FF084B075D463B43CC0897E602233C
:101DA800984636E7FC1AA742BF4163467F42C91AE4
:101DB800CB1B994601235D4698465EE54B07FF0815
:101DC8003B43CC0892E6DC1B6046A342B641401A6E
:101DD8007642801B8146000260D5FC1AA742BF41AB
:101DE80063467F42C91ACB1B99465D4676E5FF08D4
:101DF8004B073B43CC0867E60A00DB083A4300D1AF
:101E08006FE66246520713436246D40880221203E3
:101E1800144207D0C808104204D15D460400FB08EC
:101E280049070B435A0FDB00DB08520713435DE6F3
:101E38004B07FF083B43CC0849E6DC199C429B4111
:101E4800614489465B4299444B461B0200D431E603
:101E58004A46174B1A400123914698462AE616002F
:101E68006446203EF440A046202A05D04026644619
:101E7800B21A944023439A465446631E9C414346F3
:101E88001C43DBE502000024002348E5DC19BC42C2
:101E9800BF41614489467F42B94438E74B462343F2
:101EA80000D19FE606E6C046FE070000FF070000D7
:101EB800FFFF7FFFFF084B073B43CC0816E662464F
:101EC800DB08520713436246D408802212031442E7
:101ED80007D0C808104204D15D460400FB08490732
:101EE8000B435A0FDB005207DB081343FEE50023C0
:101EF800014A1C0013E5C046FF07000070B5050045
:101F08000C481C0316005B000A034900120B490D1C
:101F1800240B5B0D814208D0064A0020934203D16E
:101F280020003043431E984170BD01202A43FBD155
:101F3800F2E7C046FF0700000A0030B5134C530013
:101F480009030500090B00205B0DD20FA34204DD35
:101F58000F48834202DD0F4BD01830BD802040036C
:101F680001430D48C01A1F2808DD0C48C31AD94080
:101F78000B005842002AF0D11800EEE7084CC54083
:101F8800A446634499400B002B43F2E7FE0300008C
:101F98001D040000FFFFFF7F33040000130400004E
:101FA800EDFBFFFF70B5002816D0C317C5185D40BC
:101FB800C40F280000F04CF8114A121A0A2816DC3F
:101FC80003002E0015339E400B23181AC5405205F6
:101FD8002D032D0B530D03E00024002300250026BC
:101FE8001B052B43E40723433000190070BD0B3851
:101FF800854052052D0300262D0B530DF0E7C046F2
:102008001E04000010B5041E10D000F021F80F4B7C
:102018001B1A0A2811DC0B222100121AD140153094
:102028000A035B058440120B5B0D01E000230022CC
:102038001B0513432000190010BD22000B388240F5
:102048005B0512030024120B5B0DF1E71E04000070
:102058001C2101231B04984201D3000C10391B0AD0
:10206800984201D3000A08391B09984201D3000994
:10207800043902A2105C40187047C04604030202EB
:10208800010101010000000000000000054B82B0C2
:102098001A6C02431A641B6C18400190019B02B031
:1020A8007047C04600100240054B82B05A6B02438D
:1020B8005A635B6B18400190019B02B07047C046A1
:1020C80000100240024BD8698006C00F7047C04616
:1020D800003801400349044A8B681A40042313431B
:1020E8008B60704700240140E8FFFF7F10B586B081
:1020F8000C22002103A802F043FB8023A0241B022A
:1021080000930123E40569460193200002330293FA
:1021180002F08AF980239B0100930023694620007E
:102128000193049302F080F906B010BD10B586B093
:102138001422002101A8A02402F022FB8023E40538
:1021480069461B022000009302F06EF980239B0170
:102158000093012301930233029300236946200070
:102168000393049302F060F906B010BDF8B50400BB
:10217800FDF7C2FF002340261D00074A0749834296
:1021880000DBF8BDE75C97625F183D70D76937429E
:10219800FCD00133F3E7C04600380140CC000020F2
:1021A800F8B506000024FFF795FF0025104F114BE6
:1021B80004219A680A42FBD1186C013F80B2FFF7EC
:1021C80021FF02000B0020002900FEF75BF9040044
:1021D8000D00FFF77FFF002FE9D13000FFF712FF56
:1021E80002000B0020002900FEF788FCF8BDC0465D
:1021F8001027000000240140F0B51D0000248BB01A
:10220800049006910792079B1B78002B02D12000AF
:102218000BB0F0BD079A01320792252B0BD0069A16
:10222800944202DB01246442F1E7049A09951355AC
:102238000134099DE7E72B00203309932B68EE69E9
:102248000193AB6800220293AB69310005930598AE
:1022580000236F68FEF7E8F8002802D0854B864E09
:102268000593069AA31C03939342DBDA002300220A
:1022780039000198FEF7DEF880231B06FB18089347
:10228800002800D108973100019A089B0598FEF7AD
:10229800D1F800286ED0049B00221D1931000023BC
:1022A80005980134FEF7C6F800285CD03C232B7053
:1022B800059B019380231B06F7182D23049A1355B9
:1022C8000026002239006D4B0198FEF7C7F8002858
:1022D80002D01E2E00D084E000223900684B0198FD
:1022E800FEF7A8F8002803D033001E3300D082E0A0
:1022F800029B032B00DC88E0300003211E30FEF730
:102308007DF84B1C0593059B5A1E9341029AD318DE
:102318000293029A039B9B18069A0233934281DA2E
:102328000024049B039A9D18029BA34277DCDB439D
:10233800029ADB171340039A0399541C9D18049AB8
:10234800E418D31820225A54022E00D871E730001E
:1023580003211E30FDF76CFF4A4B049A1B5C0235C3
:1023680013552C0065E73E2337002B70059B01931E
:102378000394A5E72E696D69002200233000290027
:10238800FEF752F800281ED130002900019A089B58
:10239800FEF764F8002816D0049B00221F193000AD
:1023A800002329000134FEF745F8002806D03E2313
:1023B8003B7080231B060196EF187EE73C230196AD
:1023C8003B702F00D4E70022002339000198FEF764
:1023D80031F80028CCD080231B06FF18631C039318
:1023E8006BE7390001980022244BFEF787FB013682
:1023F8000F00019065E73900019800221F4BFEF796
:102408007FFF013E0F00019066E7029B032B2ED150
:10241800300019001F30FDF7F1FF059173E7059BA8
:10242800A34206D1002B04D02C232B700134013594
:102438007AE7029A631C934207D139000198002277
:10244800114BFEF71FF80F00019039000198FFF7B4
:1024580073FD0A21FDF7D2FF30310198297000225F
:102468003900064BFEF74CFF0F000190DEE702240F
:10247800D9E6C0469CC94622E3A6C84600002440C7
:102488000000F03F557D00080000E03FF0B56420F3
:102498008FB002F02FF98022CC4BCD4F9A627B6926
:1024A800CC4A0021134000227B61CB4B19605A6053
:1024B8000023039301330293FFF70CFEA02380222D
:1024C800DB0592019A610023022504260193BB686B
:1024D8003342FCD1FFF7FEFD019B3C6CBF4A013340
:1024E800A4B20193934203D0BD4B9C4200D84AE169
:1024F800A0238022DB0592019A62AC4202D0022D11
:1025080000D042E10198FFF77DFD0022B54BFFF7AF
:1025180063F90022B44B04000D00FDF79FFF00286B
:1025280000D04EE1002220002900AE4BFDF782FFCB
:10253800002801D00024AB4DAC4AAD4B2000290047
:10254800FEF7DEFEAB4B049005911A685B68AA495A
:10255800A14E08684968FDF795FF02000B00049832
:102568000599FEF7CBFA32687368FDF78BFF0022F6
:1025780030607160A14B20002900FEF7C1FEA04A1F
:10258800A04BFEF7BDFEA04B0022FEF7B9FEFFF7F9
:10259800D3FC02F0AFF8029B012B07D1FA20019976
:1025A8008001A031FDF7BAFD831C0293039B013320
:1025B8000393039A029B934200D97DE71800FFF723
:1025C80021FD02000B0030687168FEF797FA8F4A08
:1025D800306071608E4BFDF72DFF002800D19CE024
:1025E800FFF784FD00240023336074600023039305
:1025F80001330293FFF76EFDA0238022DB05120250
:102608009A610023022504260193BB683342FCD15A
:10261800FFF760FD019B3C6C704A0133A4B2019343
:10262800934203D06E4B9C4200D8CDE0A023802279
:10263800DB0512029A62AC4202D0022D00D00BE1F7
:102648000198FFF7DFFC0022664BFFF7C5F8002270
:10265800654B04000D00FDF701FF002800D017E1CD
:102668000022200029005F4BFDF7E4FE002801D07E
:1026780000245C4D674A684B20002900FEF740FEA5
:102688005C4B049005911A685B686449524E08686F
:102698004968FDF7F7FE02000B0004980599FEF75C
:1026A8002DFA32687368FDF7EDFE00223060716024
:1026B800524B20002900FEF723FE594A594BFEF7DA
:1026C8001FFE514B0022FEF71BFEFFF735FC02F000
:1026D80011F8029B012B07D1FA2001998001A03142
:1026E800FDF71CFD831C0293039B01330393039A9C
:1026F800029B934200D97DE71800FFF783FC020094
:102708000B0030687168FEF7F9F9474A474BFFF745
:1027180063F830607160FFF709FD2F4C00222068D4
:1027280061680023FDF786FE002803D000220023FD
:1027380022606360656824683D493E4A3E4B0868EC
:102748004968FEF7DDFD22002B00FDF773FE002827
:1027580000D1A0E00423FA21384A0893384B0694A4
:1027680007950A920B93374C374A384B20000C9246
:102778000D93C900364A06ABFFF73EFD2000FFF770
:10278800F5FC0FB0F0BD2500A1E63248401BFFF76D
:1027980039FC04900591601BFFF734FC02000B0024
:1027A80004980599FEF7AAF9019B0400981E0D00EC
:1027B800FFF728FC02000B0020002900FDF762FE4D
:1027C800A7E60024084DB7E625001EE700040050E0
:1027D80000240140FFFEFFFFA0080020E093040052
:1027E8001B0A00000000F03F804F1241FB3F8CB2F3
:1027F800AC6BBC3E300000202000002000002440CC
:102808001FDF7F9FC103CB3E00408F40AA33CE110C
:10281800BF83AB3E0E5E51D04125BB3E2800002051
:102828007BB3D16A9D00C73E6259374D5624B23DED
:1028380008000020333333333333F33F956479E1B1
:102848007FFDC53DCC0000204850FC1873D7623F7F
:10285800C85900081C0A00001048401BFFF7D2FBAB
:1028680004900591601BFFF7CDFB02000B00049854
:102878000599FEF743F9019B0400981E0D00FFF728
:10288800C1FB02000B0020002900FDF7FBFDDEE67E
:102898000024034DEEE6034871E7C0461C0A000019
:1028A800804F1241D9590008F0B5A0248025704EF8
:1028B800704A7369E4051340736182326E4BFF32CC
:1028C800AD018DB09A626420A56101F013FF6B48D9
:1028D800FFF766FC6A4B0090019100980199A56288
:1028E8001F68684B1C68E41BFFF726FBA04208D34F
:1028F8002000FFF787FB0022634BFEF76DFF009077
:102908000191624B62491A685B6808684968FDF77B
:10291800B9FD029003912000FFF774FB0400380012
:102928000D00FFF76FFB02000B0000980199FEF7FE
:1029380053FF02000B0020002900FEF7DFF80022F9
:10294800514BFEF749FF02000B0002980399FEF76E
:10295800D5F8504B1A685B68FEF73EFF00224E4BD5
:1029680004000D00FDF77AFD00285DD0802773690B
:10297800404A7F0013401F437761FFF7B7FBA0274A
:102988008023FF051B02BB61642001F0B3FE3B48B6
:10299800FFF706FC414B04001B680D000093404BF9
:1029A8001E68009BF61AFFF7C7FAB04208D330003A
:1029B800FFF728FB0022344BFEF70EFF04000D0042
:1029C80080231B02BB623749304B086849681A6884
:1029D8005B68FDF757FD029003913000FFF712FB8B
:1029E800060000980F00FFF70DFB02000B00200007
:1029F8002900FEF7F1FE02000B0030003900FEF757
:102A08007DF80022204BFEF7E7FE02000B0002983B
:102A18000399FEF773F81F4B1A685B68FEF7DCFE34
:102A280004000D00FFF782FB00220023200029008C
:102A3800FDF700FD002801D00024002504231A4AD0
:102A480006931A4BFA2108920993002204940595DB
:102A5800174B184C0A920B93C900174A04AB200075
:102A6800FFF7CAFB2000FFF781FB0DB0F0BDC046A1
:102A780000240140FFFEFFFF000400501027000063
:102A880018000020100000200000F03F3000002057
:102A9800200000203800002000C8A9401C000020A9
:102AA80014000020280000207B14AE47E17A843F00
:102AB800389C7C41CC000020EB590008F0B54D4C07
:102AC8004D4D6369A0272B40636180234B4EFF0562
:102AD8009B01A3B0BB61642001F00CFE3000FFF73E
:102AE8005FFB80239B0100900191BB62642001F091
:102AF80001FE009801990022414BFDF7C3FCFFF746
:102B08001BFA404B18603000FFF74AFB00223C4B91
:102B1800FDF7B8FCFFF710FA3B4B18608023626999
:102B28005B002A4013436361FFF7E0FA80231B022E
:102B3800BB61642001F0DEFD3000FFF731FB80232C
:102B480004000D001B02BB62642001F0D3FD0022CB
:102B58002B4B20002900FDF795FCFFF7EDF92B4FD3
:102B6800002438603000FFF71BFB0022244BFDF7E0
:102B780089FCFFF7E1F9264E00253060FFF7D6FA09
:102B8800204B1868FFF73EFA042302900391386837
:102B980006940795089409950493FFF733FA0427D8
:102BA800194B0A900B9118680E940F951094119573
:102BB8000C97FFF727FA129013913068169417951F
:102BC800189419951497FFF71DFA1A901B91FA217A
:102BD8001E941F95209421950E4C0F4A02ABC900F4
:102BE80020001C97FFF708FB2000FFF7BFFA23B06F
:102BF800F0BDC04600240140FFFEFFFF1027000083
:102C08000000E03F10000020180000201400002001
:102C18001C000020CC000020FA590008F0B5A024C0
:102C280080258027664A67495369674E0B40E4054B
:102C3800AD0197B053616420B762A56101F05AFDF8
:102C48006248FFF7ADFA624B02900391A5621B68D8
:102C580060490093604B086849681A685B68FDF72B
:102C680011FC5E4B04001868009B0D00C01AFFF7AA
:102C7800C9F9049005910098FFF7C4F902000B0008
:102C880002980399FEF7A8FD02000B000498059925
:102C9800FDF734FF0022524BFEF79EFD02000B00A9
:102CA80020002900FDF72AFF0023002204000D0060
:102CB800FDF7C0FB4B4B002800D076E01C605D6040
:102CC800B761642001F016FD4048FFF769FA434BED
:102CD80002900391B7621C683D4B3E491B68086827
:102CE800496800933C4B1A685B68FDF7CBFB009B77
:102CF8000600E01A0F00FFF785F9049005912000FF
:102D0800FFF780F9040000980D00FFF77BF9020037
:102D18000B0002980399FEF75FFD02000B002000EC
:102D28002900FEF759FD02000B0004980599FDF7EC
:102D3800E5FE00222A4BFEF74FFD02000B00300093
:102D48003900FDF7DBFE0023002204000D00FDF72B
:102D580071FB254B00282DD11C605D601E685F68E3
:102D68000020204A214C1168526806910792204998
:102D780004220C900D9114901591FA211D4D089282
:102D88000A940B95129413951B4C109206AB1B4A90
:102D9800C9002000009601970E960F97FFF72CFAAE
:102DA8002000FFF7E3F917B0F0BD002100221960F9
:102DB8005A6085E70021002219605A60CEE7C046B4
:102DC80000240140FFFEFFFF000400501027000010
:102DD80018000020200000203000002010000020F3
:102DE8000000F03F38000020400000207B14AE4770
:102DF80000408F40E17A843FCC0000200C5A000844
:102E0800F0B5214C214A636991B013406361802277
:102E1800A0239201DB059A61FFF75CF90423A268FD
:102E28001A42FCD1A0238022DB059201256C9A620C
:102E3800FFF750F90426ADB2A3683342FCD128004D
:102E4800FFF7E0F8276C0025002400900191B8B244
:102E580004940595069407950296FFF7D3F8089011
:102E68000991FA210C940D950E940F95084C6B4618
:102E7800084AC90020000A96FFF7BEF92000FFF7AC
:102E880075F911B0F0BDC04600240140FFFEFFFFF8
:102E9800CC000020275A0008F0B5A0248025802601
:102EA800E64AE7495369E74FFDB00B40E405AD0139
:102EB800169053616420BE62A56101F01BFCE248D4
:102EC800FFF76EF900900191BE616420A56201F0E0
:102ED80011FCDD48FFF764F9DC4B02900391BE62F8
:102EE800A5621868FFF78EF804000D00D84B186823
:102EF800FFF788F822002B00FEF76EFC06000F0093
:102F08000098019922002B00FEF766FC32003B0076
:102F1800FDF7F4FDCF4AD04BFEF7F2F922002B0063
:102F28000090019102980399FEF756FC32003B008D
:102F3800FDF7E4FD02000B000020C849FEF74CFC39
:102F4800C44AC54BFEF7DCF9C54B0F001A685B682D
:102F5800C449060008684968FDF794FA009A019B7D
:102F680004000D00BB48BC49FEF736FC22002B00CC
:102F7800FDF7C4FDBC4B029003911A685B68FEF72D
:102F8800BFF902000B0000980199FEF725FC3200FA
:102F9800069007913B00AF48AF49FEF71DFC2200A1
:102FA8002B00FDF7ABFD04900591B04B1A685B68E8
:102FB800FEF7A6F902000B0030003900FEF70CFC02
:102FC800002208900991029803990023FDF732FA2C
:102FD800002803D00023002402930394069807993D
:102FE80000220023FDF726FA002803D0002300243E
:102FF800069307940498059900220023FDF71AFA0E
:10300800002803D000230024049305940898099904
:1030180000220023FDF70EFA002803D00023002425
:1030280008930994642001F065FBA0268027864850
:10303800FFF7B6F88023834AF605BF010A900B9183
:1030480093616420B76101F055FB7F48FFF7A8F84A
:103058007E4BB762040018680D00FEF7D3FF02002C
:103068000B00009001910A980B99FEF7B5FB784B7D
:103078000A900B911868FEF7C5FF22002B00060086
:103088000F00FEF7A9FB0022794B04000D00FDF7A5
:10309800F9F90A9A0B9BFDF7CDF9002800D121E236
:1030A800009A019B30003900FEF796FB02000B00E6
:1030B8000A980B99FDF722FD664A674BFEF720F93F
:1030C80012901391674B80255C681B6818931994BC
:1030D800634B80265C681B681A931B94FFF706F8FD
:1030E8005649574B4A69A0241A408023554F5B0024
:1030F8001343E4052D024B616420BE62A56101F013
:10310800F9FA5148FFF74CF800900191BE6164202C
:10311800A56201F0EFFA4C48FFF742F8554B0A90C8
:103128000B91BE62A5621868FEF76CFF04000D00E3
:10313800514B1868FEF766FF22002B00FEF74CFB88
:1031480006000F000098019922002B00FEF744FBAF
:1031580032003B00FDF7D2FC3E4A3F4BFEF7D0F869
:1031680022002B00009001910A980B99FEF734FB7E
:1031780032003B00FDF7C2FC02000B00002037497B
:10318800FEF72AFB334A344BFEF7BAF8344B0F00EC
:103198001A685B683949060008684968FDF772F9DA
:1031A800009A019B04000D002A482B49FEF714FBE6
:1031B80022002B00FDF7A2FC2B4B0E900F911A68F2
:1031C8005B68FEF79DF802000B0000980199FEF776
:1031D80003FB32000A900B913B001E481E49FEF784
:1031E800FBFA22002B00FDF789FC109011911F4B70
:1031F8001A685B68FEF784F802000B00300039009B
:10320800FEF7EAFA00220C900D910E980F99002310
:10321800FDF710F9002803D0002300240E930F9423
:103228000A980B9900220023FDF704F9002827D0FB
:10323800002300240A930B9422E0C0460024014096
:10324800FFFEFFFF000400501027000018000020B8
:10325800100000206666666666660A400000F03F59
:10326800300000202000002038000020400000200E
:10327800000032401C00002014000020280000201C
:103288001098119900220023FDF7D4F8002803D0E4
:1032980000230024109311940C980D990022002308
:1032A800FDF7C8F8002803D0002300240C930D94E0
:1032B800642001F01FFAA0248025A948FEF770FFBA
:1032C8008022A84BE4052D02149015919A61642080
:1032D800A56101F00FFAA248FEF762FF8022A14B18
:1032E80006009A62A5620F00FEF720FF9E4B186841
:1032F800FEF788FE02000B000090019114981599C2
:10330800FEF76AFA994B040018680D00FEF77AFE7A
:1033180032003B0014901591FEF75EFA0022944BA0
:1033280006000F00FDF7AEF822002B00FDF782F82B
:10333800002800D1F6E0009A019B14981599FEF731
:103348004BFA02000B0020002900FDF7D7FB894A41
:10335800894BFDF7D5FF04000091884B88491A680E
:103368005B6808684968FDF78DF802000B002000CB
:103378000099FDF7C3FB834A0D0014901791824B07
:103388000C980D99FDF76AF8002800D116E1069807
:1033980007997C4A7C4BFDF74DF8002800D10DE1D8
:1033A8000022002320000099FDF73EF8002800D1F4
:1033B80004E1169B002B00D000E10A9A0B9B0698AB
:1033C8000799FEF709FA040002000B000D000698A1
:1033D8000799FDF793FB02000B000E980F9901F077
:1033E8000DFA220006000F000A980B992B00FDF732
:1033F80085FB02000B000298039901F0FFF9020017
:103408000B0030003900FDF779FB02000B000600C5
:103418000F0002980399FDF771FB00225B4BFDF743
:1034280031F801F0B5F9069B079C594A1C931D9485
:10343800584B009001912092219300220023229260
:1034480023930299039A249125925349534A0023BE
:103458002891299200222A922B930A990B9A4D4B74
:103468002C912D924A4A0424309231930022002351
:10347800329233930E990F9A494B349135920098B2
:103488000199484A1E9438923993002200233A92AF
:103498003B93454A454B26942E943694FDF730FFCE
:1034A80002000B0006980799FDF728FB002200236D
:1034B8003C903D9144964597409241934292439364
:1034C800489249934A924B93394A3E9446941CAB8E
:1034D800FA213848C900FEF78FFE3648FEF746FE47
:1034E8007DB0F0BD00220A980B99214BFCF7CAFF6A
:1034F80022002B00FCF79EFF00280ED0009A019BAB
:1035080030003900FEF768F902000B00200029009E
:10351800FDF7F4FA174A284BD0E50023002412934C
:103528001394CFE500222000114B2900FCF7AAFFD5
:1035380032003B00FCF77EFF041E0ED0009A019B70
:1035480014981599FEF748F902000B00300039006D
:10355800FDF7D4FA074A184BFBE60090FDE6C04693
:1035680010270000000400501C0000201400002058
:10357800000032406666666666660A4030000020D3
:10358800280000203D0AD7A3703D0A400000F03F04
:10359800FCA9F1D24D62503F54E41071732AD93E10
:1035A8002B1B703E2B69A4296B6B09CE200B9A3F0D
:1035B800325A0008CC00002066660AC0C34AC44BD1
:1035C8000A980B99FCF74AFF002800D1A1E0089857
:1035D8000999BE4ABE4BFCF72DFF002800D198E0A0
:1035E8000022002320000099FCF71EFF002800D1CC
:1035F8008FE0169B002B00D0C4E10C9A0D9B089815
:103608000999FEF7E9F8040002000B000D0008987C
:103618000999FDF773FA02000B001098119901F04F
:10362800EDF8220006000F000C980D992B00FDF70D
:1036380065FA02000B000498059901F0DFF8020012
:103648000B0030003900FDF759FA02000B000600A4
:103658000F0004980599FDF751FA00229D4BFCF7DD
:1036680011FF01F095F8089B099C9B4A1C931D9437
:103678009A4B0090019120922193002200232292DC
:1036880023930499059A249125929549954A0023F4
:103698002891299200222A922B930C990D9A8F4BEC
:1036A8002C912D928C4A04243092319300220023CD
:1036B800329233931099119A8B4B3491359200982A
:1036C80001998A4A1E9438923993002200233A922B
:1036D8003B93874A874B26942E943694FDF710FE29
:1036E80002000B0008980999FDF708FA0022002348
:1036F8003C903D9140924193429243934892499322
:103708004A924B93449645977B4A3E9446941CAB09
:10371800DEE60022002320000099FCF79FFE002827
:1037280042D0169B002B00D03EE1109A119B1C92B0
:103738001D9300220023229223932200009B664CB3
:1037480024922593002200232A922B93149A179BE4
:10375800624D2C922D93002200230426329233933B
:1037680028942995389439951C0013005F485E49C0
:103778003A933B9420902191309031910698079983
:10378800349035910299039A3C913D92554A544997
:1037980042934394409141921E96584A26962E96FB
:1037A80036963E961CAB93E6002200232000009933
:1037B800FCF740FE002848D0169B002B00D0F3E011
:1037C8000E9A0F9B1C921D93802248484649120668
:1037D8002090219100200021944622902391009965
:1037E8003E4A614425913C490020289129920021B4
:1037F800149A04262C926246030024940C002A9002
:103808002B9139493948AD18309031910899099A66
:10381800349135923049314A329333943891399200
:103828000499059A3C913D922E4A2D493A933B942E
:103838004091419242934394314A1E9626962D9583
:103848002E9636963E961CAB42E6002200232000B8
:103858000099FCF7E9FD002800D1A5E00C980D9926
:103868000022284BFCF7FAFD002853D00E980F9938
:10387800254A264BFDF744FD069A079BFDF740FDB8
:103888000A9A0B9BFDF73AF9029A039BFCF7E6FDAF
:1038980000283FD002980399114A124BFCF7DEFD2D
:1038A800002837D0169B002B34D1029B039C1C9315
:1038B8001D9404230B4C1E93094B154A2093219405
:1038C80000230024229323941CAB01E63D0AD7A3CE
:1038D800703D0A400000F03FFCA9F1D24D62503F14
:1038E80054E41071732AD93E2B1B703E2B69A4290E
:1038F8006B6B09CE200B9A3F285B00081E5C000802
:10390800155D000800000840CDCCCCCCCCCCEC3FF9
:103918000B5E000800220A980B996A4BFCF79EFD83
:10392800002841D010981199674A684BFDF7E8FCC8
:10393800089A099BFDF7E4FC0C9A0D9BFDF7DEF84D
:10394800049A059BFCF78AFD00282DD00498059958
:103958005F4A604BFCF782FD002825D0169B002BA0
:1039680022D1049B059C1C931D940423594C1E933F
:10397800574B594A209321940023002422932394DF
:103988001CABA5E50022002320000099FCF766FD8A
:10399800002800D062E70022002320000099FCF7ED
:1039A80049FD002800D150E7069A079B0020002116
:1039B80004251C921D93029A039B24922593444A42
:1039C800444B464E289229930A9A0B9B2C922D938E
:1039D8000E9A0F9B34923593414A424B424F2290A4
:1039E80023912A902B913290339138923993129ADD
:1039F800139B3A903B913C923D931A9A1B9B4290A1
:103A080043911898199920962197309631974096A6
:103A180041971E9526952E9536953E95FCF732FDD5
:103A280002000B0012981399FDF768F8284A294BF1
:103A38004490459148924993220000200021009B20
:103A4800284C4C924D93149A179B4A904B91549240
:103A58005593234B529053915893599403000C005B
:103A68000C990D9A1E485C915D921099119A649177
:103A780065921C495A935B9462936394154A5096D5
:103A880051976096619746954E9556955E956695C1
:103A980068906991089809996C906D9104980599B6
:103AA800749075910A496A936B94729373947891A0
:103AB80079927A937B94709671970C4A6E95769565
:103AC8001CAB05E500000840CDCCCCCCCCCCEC3F01
:103AD80054E41071732AD93E015F0008FCA9F1D2A1
:103AE8002B69A4292B1B703E4D62503FF75F0008DD
:103AF8008022F0B5424E52007369A02713437361C8
:103B08008023FF059B01BB62FA23002400258BB0AC
:103B18009B000093FEF7DEFA80239B01BB61042320
:103B2800B2681A42FCD1306C80B2FEF76BFA020020
:103B38000B0020002900FCF7A5FC80239B01BB6239
:103B4800040001200D0000F0D5FD009B013B00930F
:103B5800002BDFD1002220002A4B2900FCF7CEFFE2
:103B6800294B06001C68294B0F001B68E41A20002B
:103B7800FEF748FA0090019130003900FEF7DCF9B1
:103B8800A04207D3009801990022214BFDF724FE9B
:103B980006000F001F4B20491A685B6808684968CF
:103BA800FCF770FC320004000D00009801993B00FE
:103BB800FCF7A4FF0022164BFDF70EFE02000B00D7
:103BC80020002900FCF79AFF144B00241A685B6850
:103BD800FDF702FE04230493002302900391FA21C7
:103BE80006930794089309940D4C0E4A02ABC9003A
:103BF8002000FEF701FB2000FEF7B8FA0BB0F0BD7D
:103C08000024014000408F401000002018000020D0
:103C18000000F03F30000020200000203800002085
:103C2800CC000020ED60000810B50248FEF79EFAAF
:103C380010BDC046FA600008012210B5024B0348C7
:103C48001A70FEF793FA10BD000000208B6500087B
:103C580010B50248FEF78AFA10BDC0461C6A000873
:103C680010B50A48FEF782FA0024FEF72BFA00285E
:103C780002D0074B5C6AE4B20648FEF777FAFEF713
:103C880013FE702CF1D1FFF7E3FF10BDAD6E0008F5
:103C9800003801403E73000810B50A48FEF766FA7E
:103CA8000024FEF70FFA002802D0074B5C6AE4B242
:103CB8000648FEF75BFAFEF7E9FB702CF1D1FFF737
:103CC800C7FF10BD46730008003801403E73000866
:103CD80070B500250C48FEF749FA2C000126FEF7BE
:103CE800F1F9002802D0094B5C6AE4B2752C00D1C6
:103CF80035000748FEF73AFA2800FFF7CDF8702C90
:103D0800EDD1FFF7A5FF70BDD77700080038014057
:103D18003E730008F0B55F4893B0FEF727FAFEF748
:103D2800D1F90028FBD001245B4E756AEDB20D2D48
:103D380060D15A4F3800FEF719FA002301220A20F1
:103D480057490193012C00D072E05648FEF70EFA4D
:103D5800FEF7B8F90028FBD02500736ADBB20093A0
:103D6800009B0D2B00D06CE03800FEF7FFF9002314
:103D780001220A204A490093012D00D081E00198D0
:103D8800FEF740F904000D00474B00981C605D6089
:103D9800FEF738F9454B0A900B91186059600323D8
:103DA8009C46614602940395002400220C91FA2156
:103DB8003F4D0493089409953E4B10941195384C47
:103DC800069207930E920F93C9003B4A02AB20005C
:103DD800FEF712FA2000FEF7C9F93848FEF7C6F9CF
:103DE800FEF770F90028FBD03800736AFEF7BEF9B9
:103DF80013B0F0BD02AB1D70002302AA537010006F
:103E0800FEF7B4F92B00303B092B09D8244B1D557C
:103E18000134FEF757F90028FBD0756AEDB286E742
:103E28002748FEF7A3F92748FEF7A0F90124F0E791
:103E3800013C0B5D019D303B5343EB18424301931A
:103E480080E7009A02AB1A70002218005A70FEF739
:103E58008DF9009B303B092B0BD8114B009A5A5512
:103E68000135FEF72FF90028FBD0736ADBB2009307
:103E780076E71348FEF77AF90A48FEF777F925003E
:103E8800EFE7013D4B5D009C303B5343E318424351
:103E9800009371E7687C000800380140CC7C00087A
:103EA800CC000020CE7C0008200000202800002044
:103EB80060E346410000F03FF87C00080E7D0008F2
:103EC8009B7C0008727C000807200223274A10B553
:103ED800116881430B43136013680340022BFBD125
:103EE8008022234B520019680A431A608022D200AC
:103EF80019681142FCD0DA681E4911401E4A0A436B
:103F0800DA608022D96852020A43DA60DA681B490B
:103F180011401B4A0A43DA608022196852040A4396
:103F28001A608022D96852050A43DA608022920416
:103F380019681142FCD09A6812490A4007219A6010
:103F48009A688A43110002220A4338219A609A68C3
:103F58000A40102AFBD19A680B490C480A409A601B
:103F680000F0B8FB094800F0DBFB10BD0020024060
:103F7800001002408C80C1FF021406008C80FF1FD5
:103F880002140080FFF0FFFFFF8FFFFF0090D003B7
:103F9800F0B5012095B0FEF779F88021D44F490596
:103FA800FA6B10260A43FA63C022FB6B12060B4019
:103FB800D0490193019B0B6AA0251B021B0A1343DE
:103FC80008220B62CC4B00241968ED050A431A60DD
:103FD8001A6832431A60FFF777FF182200210CA8ED
:103FE80000F0CEFB0220FEF75FF80120FEF75CF838
:103FF80080228023C148920183620CA9AA620C9393
:104008007F3B0D930E940F94109400F00DFA8022CC
:10401800920101230C9203220CA928000E920D9301
:104028000F94109400F000FA80230CA91B022800BA
:104038000C930D94109400F0F7F93200210002A8B7
:1040480000F09EFB80262100182206A800F098FBAD
:10405800210018220CA800F093FB80207B6DF60548
:104068009B009B0833437B654003FEF70FF8012054
:10407800FEF71AF8012303220CA928000C930D92CD
:10408800109400F0D1F90394049405949C4C02A96F
:104098002000029600F082F98022E368920313431D
:1040A800E3608022236892011342FAD0F023226051
:1040B80007938023002501265B0106A990480695F1
:1040C800089509950A950B9300F084F923698D4AA0
:1040D800B343236123697021134007222361636975
:1040E8000CA89343033A1343636163690B43636109
:1040F8006368290093436360636804329343636091
:10410800A368814A1A4080235B0513430F22A360EA
:10411800A36A9343A36263697C4A134022326361B2
:10412800FF3200F02DFB2900182206A800F028FB1A
:10413800032280207B6DC00193437B65FDF7A6FFBA
:104148003000FDF7B1FF8023A02002279B0006A9BD
:10415800C0050693089509950A9507970B9600F0F0
:1041680063F98023A020DB0006A9C0050693089503
:1041780009950A9507970B9600F056F9E1235B021B
:104188000D930C230C950E950F951095129513957C
:104198005F4D0CA92800119300F02EFAEFF310825E
:1041A80086F31088AB68DB00DB08AB6082F310880D
:1041B800EFF3108286F310885649AB680B40AB606A
:1041C80082F310884F4A2B68802113402B606B685C
:1041D800514A890313402A226B60AB689343AB6052
:1041E8002B681E4380232E60DB03EA690A42FCD059
:1041F800EA691A42F9D08022A168484812060140AB
:104208000A43A260A368002BFCDB0126A368FA27F7
:10421800034033436420A36000F06CFAFF00FDF70D
:1042280051FF3F4C00280AD0686AC0B2002806D067
:104238002278002A16D070280AD076280DD0237844
:10424800002BECD0FFF7F0FC380000F053FAE6E75B
:1042580000232370FFF7F0FCF1E700232370FFF73A
:1042680059FDF7E72F4B1978002920D070281AD06C
:10427800732812D06F28E2D12B48FDF777FFFEF79D
:104288001DFC2A48FDF772FFFEF700F9284B186855
:104298005968284B18605960D1E72748FDF766FF31
:1042A800FEF7BCFCCBE71A70FFF7D2FCC7E765281E
:1042B80009D86028C3D961380428C0D8FBF724FF7F
:1042C8000FBF09121500722806D07528B7D12670BD
:1042D800B5E7FFF7E1FCB2E7FFF7C2FCAFE7FEF78F
:1042E8008FFDACE7FFF7F4FCA9E7FFF701FCA6E7B1
:1042F8000010024000ED00E0000001400004005002
:1043080000240140FFFFFFDFE8FFFF6FFFFEFFFF14
:1043180000380140FFFFFFF1FFB7FFFFE8FFFF7F15
:1043280001000020000000203D7D0008457D0008B8
:10433800A0080020080000204D7D0008FEE7FEE7E9
:1043480070477047704770470D488546FFF7FBFF79
:104358000C480D490D4A002302E0D458C4500433D8
:10436800C4188C42F9D30A4A0A4C002301E01360AE
:104378000432A242FBD300F0DFF9FFF709FEFEE7A3
:104388000020002000000020B0000020387E000837
:10439800B0000020A8080020FEE7000082680300A3
:1043A80030B5012014000440024210D18D684A68DB
:1043B800D8682A43CD6809682A43054D2840024336
:1043C8002000DA601A69920092080A431A6130BD27
:1043D800C73FFFFFC3680200C3688368012070B548
:1043E80003421BD1CC680B68D06823430E694D6922
:1043F8000C4C800202D54868F02810D033432B4378
:10440800D0688D6820402B430343D360D3680020D5
:104418009B0203D5936A49680B43936270BDD068C9
:104428003343EFE73CC2FEFFF7B5020000270C68F4
:104438002000F84000D1FEBD01202300B840034011
:10444800044233D04868032484461800654658431C
:104458004443013DE443012D0BD88D6896684543DC
:1044680026403543CE6895605E4355689D43354385
:1044780055600D69D668454326403543D560654685
:10448800022D0DD14D690195FF2B11D803000F2581
:1044980043435D43166AAE43019D6B431E43166258
:1044A8001368234064466043034313600137BEE743
:1044B8000F261B0A5B435B435E43556AB543019E67
:1044C80073431D435562EBE7054B064A9B681B0582
:1044D8001B0F9B009B581F221340D8407047C046B3
:1044E800001002406C7D0008054B064A9B685B047F
:1044F8005B0F9B009B581F221340D8407047C04653
:1045080000100240AC7D00083821154B10B59A68A0
:104518000A40082A21D0102A19D1D8680D3A10402B
:104528000338421E90410F4A404210408018DA6812
:10453800D968DC68490653045B0E490F01315843BA
:10454800FBF7ECFD610F0131FBF7E8FD10BD1B68BF
:1045580005489B045B0FD840F8E70248F6E7C046D9
:104568000010024000127A000024F40010B5040084
:10457800FFF7CAFF2060FFF7A7FF6060FFF7B4FFEF
:10458800A06010BD030010B50020032B10D1154A00
:10459800506D0340C02080021843134B984208D046
:1045A800124B98420ED0124B984214D1FFF7ACFF31
:1045B80010BD126880231000DB0018401A42F7D0A3
:1045C8000C48F5E7D26D0223100018401A42EFD0CC
:1045D80080200002ECE7FFF797FFFFF775FFFFF772
:1045E80083FFE5E700100240020003000300030018
:1045F800010003000024F400F0B50126036804005C
:104608000D0085B0334248D18B68096902680B43B5
:1046180069690B43E9690B4327490A40134303605F
:104628004368264A1340EA68134343608368244A70
:104638001340AA6913438360224B984222D1032076
:10464800FFF7A0FF002820D06F68002F1DD02B682F
:1046580000260B2B1AD81C4A9B009958FBF75EFDC5
:104668008022E9697B08120291421ED14000C018DD
:104678003900FBF753FD154B03400007400F184363
:10468800E06003E0124B98420AD001260F22E16A4B
:104698002B6891439BB20B43E362300005B0F0BD39
:1046A80001A8FFF763FF0398CCE73900C018FBF7B0
:1046B80035FD80B2E4E7C046F369FFEFFFCFFFFFA7
:1046C800FFFCFFFF00380140CC7D0008F0FF000030
:1046D80000440040FA2110B58900FBF71FFD0022B5
:1046E800034B013858609A6005321A6010BDC04605
:1046F80010E000E0094A82B013680193019B431C53
:10470800591E8B41C01880235B02002801D102B0DA
:10471800704711681942F8D00138F6E710E000E058
:10472800014B18607047C04648000020014B1868CC
:104738007047C0464C00002070B500260C4D0D4C4B
:10474800641BA410A64209D1002601F0EBF80A4D1B
:104758000A4C641BA410A64205D170BDB300EB58E7
:1047680098470136EEE7B300EB5898470136F2E771
:10477800307E0008307E0008307E0008347E000855
:1047880003008218934200D1704719700133F9E78A
:10479800F8B504000D0000F09FF8220006000F0095
:1047A8002B0020002900FDF7A9FB002815D10022C5
:1047B800002320002900FBF751FE00280DD100221C
:1047C800002320002900FBF72FFE002808D0FFF760
:1047D800ADFF22230026074F036030003900F8BDE3
:1047E800FFF7A4FF21230360034801F021F8060026
:1047F8000F00F2E70000F0FFCD7C0008F7B51400C9
:104808001D000090019100F017FA220006000F0029
:104818002B0020002900FDF771FB00283FD10098EC
:10482800019900220023FBF7FFFD002819D0002280
:10483800002320002900FBF7F7FD002846D12000BF
:10484800290000F0EDFF002829D0002200232000D5
:104858002900FBF7EFFD002821D0FFF767FF22238F
:104868001CE03000390000F0DBFF00281BD1009865
:10487800019900F0D5FF002815D02000290000F08C
:10488800CFFF00280FD032003B0030003900FDF781
:1048980035FB0028E1D0FFF749FF212303603000F2
:1048A800390003B0F0BD0022002330003900FBF7C7
:1048B800BBFD0028F3D00098019900F0B1FF002853
:1048C800EDD02000290000F0ABFFC4E70026014F1F
:1048D800E5E7C0460000F03F8022F0B50B008DB040
:1048E8005203914222DA4A005208024307D10022B9
:1048F80000230020B349FCF701F90DB0F0BD0029F1
:1049080005DA0200FCF768FF00220023F3E7AE4B4C
:104918000022FCF7F5FC36240B006442AB4A9342B4
:1049280006DD02000B00FBF7ADFDE6E70024F5E726
:10493800A74D1A15521912191B03A64C1B0B0293EB
:104948001C1980235B032340A34C029D5C401B156C
:104958009B1825430022009329009F4BFCF73CFF3E
:10496800029B060002331B030F0000221B0B022BC5
:1049780064DC0023FBF758FD002819D0009B002BAE
:1049880000D11CE11800FDF70DFB944A944B04007C
:104998000D00FCF7B5FC934A06000F00924B20006F
:1049A8002900FCF7ADFC02000B0030003900BAE723
:1049B8008E4A8F4B30003900FCF7A2FC02000B0036
:1049C80000208C49FCF708FF320004000D003B0072
:1049D80030003900FCF794FC0B000200290020008D
:1049E800FCF78EFC009B02900391002B06D102007D
:1049F8000B0030003900FCF7EFFE7EE70098FDF76A
:104A0800D1FA764A764B04000D00FCF779FC754A1A
:104A180000900191744B20002900FCF771FC020002
:104A28000B0002980399FCF7D7FE32003B00FCF715
:104A3800D3FE02000B0000980199DCE78023DB0518
:104A4800FBF720FD02000B0030003900FCF756F898
:104A5800049005910098FDF7A5FA049A059B069025
:104A6800079110001900FCF74BFC634A029B94461F
:104A7800634402000B930B0008900991FCF740FC7B
:104A880004000D005D4A5E4BFCF73AFC5D4A5E4B44
:104A9800FBF7F8FC22002B00FCF732FC5B4A5C4B6E
:104AA800FBF7F0FC22002B00FCF72AFC594A5A4B72
:104AB800FBF7E8FC089A099BFCF722FC574A089088
:104AC8000991574B20002900FCF71AFC554A564B10
:104AD800FBF7D8FC22002B00FCF712FC534A544B7E
:104AE800FBF7D0FC22002B00FCF70AFC02000B00AD
:104AF80008980999FBF7C6FC029A4E4B04009B1ACA
:104B08000B9A0D001343002B34DD0022394B300083
:104B18003900FCF7F5FB32003B00FCF7F1FB020023
:104B28000B000290039120002900FBF7ABFC049ACC
:104B3800059BFCF7E5FB009B04000D00002B06D14C
:104B480002000B0002980399FCF746FE4FE7234A40
:104B5800234B06980799FCF7D3FB224A0090019152
:104B680006980799204BFCF7CBFB22002B00FBF79C
:104B780089FC54E702000B0030003900FCF72CFEDA
:104B8800049A059BFCF7BCFB009B04000D00002B5E
:104B980002D102000B002CE7104A114B0698079926
:104BA800FCF7AEFB0F4A00900191069807990E4B4F
:104BB800FCF7A6FB02000B002000290033E70020C9
:104BC80000219AE6000050C300005043FFFFEF7F2A
:104BD80001FCFFFF645F09000000F03F0000E0FEF9
:104BE800422EE63F763C7935EF39EA3D5555555525
:104BF8005555D53F0000E03F86EBF9FF44523EDFB4
:104C080012F1C23FDE03CB966446C73F5993229404
:104C18002449D23F935555555555E53F9FC678D001
:104C2800099AC33FAF788E1DC571CC3F04FA979996
:104C38009999D93F51B80600F0B595B002920393FF
:104C4800039B039A0493029B56001A0076080700F8
:104C58000D00324319D180210903694002000B007D
:104C680092185B4189498B4206D801D000F0B6FC06
:104C7800002A01D100F0B2FC029A039B38002900F7
:104C8800FBF700FC00900191ADE0814A4C000891CF
:104C980000906408944208DC01D10028ECD17C4AD9
:104CA800964202DC0CD1002B0AD07A4BEB183B431E
:104CB800E2D180210398090348400300029ACFE714
:104CC80000220692002D69DA734A964264DC734A20
:104CD800964211DD724932155218142A3CDD3421EE
:104CE8008A1A0299D14008009040984204D10122C2
:104CF80011409218521A0692002B3CD03800290015
:104D080000F08BFD00900191002F00D094E0002C62
:104D180005D0644AAB009B08934200D08CE0049B0A
:104D2800002B07DA009A019B00205E49FBF7E6FE9C
:104D380000900191089B002B55DA564BE418069B0E
:104D48001C4300D06CE0009A019B10001900FCF78E
:104D580043FD02000B001CE0002BCFD114339A1A3C
:104D68003300134119009140B14204D1012213408C
:104D78009218D31A06934B4B9E4238D1380029001B
:104D8800049B00900191002B2DDA3A002B000020A3
:104D98004449FBF7B3FE75E702220692002BADD11A
:104DA8003B4B9E42E7D13B4BE3181F4301D100F038
:104DB80015FC3A4B9C4209DD049B002B01DA00F0FC
:104DC80011FC029B039C009301940CE0049B002BB4
:104DD80001DB00F007FC802212069446029B009338
:104DE800039B634401930098019915B0F0BD80239B
:104DF800049ADB059A4206D13A002B0038002900B4
:104E0800FCF77EFA3EE7284B049A9A4200D075E7F1
:104E1800002D00DA72E73800290000F017FC31E7AE
:104E2800069B012BDFD1009880210200019809061A
:104E3800431800920193D6E7EB0F013B0E930E9AAD
:104E4800069B134304D13A002B00380029007EE763
:104E5800164B9E4200DCEFE0154B9E4209DD0F4BDE
:104E68009C420CDC049B002B0CDA002000F0CEFCEA
:104E780008E7104B9C42F5DD0A4B9C421CDD049B65
:104E8800002BF2DC002000F0BAFCFBE60000F0FF8B
:104E98000000F07F000010C0FFFF3F43FFFFEF3F1F
:104EA80001FCFFFF0000F03F0000E03F0000E04190
:104EB8000000F043FEFFEF3F002200980199524B9B
:104EC800FCF78AFCC022514BD20504000D00FCF708
:104ED80017FA4F4A009001914E4B20002900FCF729
:104EE8000FFA0022049005914B4B20002900FCF793
:104EF80007FA02000B0049484949FCF76DFC2200FB
:104F08002B00FCF7FDF902000B0000204549FCF7D7
:104F180063FC220006000F002B0020002900FCF78C
:104F2800EFF902000B0030003900FCF7E9F93E4ABE
:104F3800364BFCF7E5F902000B0004980599FCF7DD
:104F48004BFC02000B0004000D0000980199FBF7D0
:104F580099FA009A019B00200F000600FCF73CFC20
:104F680002000B0020002900FCF736FC069B0E9A75
:104F7800013B04900591134300D0DBE100232B4C47
:104F880000930194029C039D0298039900242B002E
:104F98002200FCF721FC32003B00FCF7B1F9029A31
:104FA800039B0690079104980599FCF7A9F902005C
:104FB8000B0006980799FBF765FA22002B0004906E
:104FC800059130003900FCF79BF906000F000B0033
:104FD80002000498059906960797FBF753FA144BB5
:104FE80005000C000891994200DCD6E2114BCB1861
:104FF800034300D1D8E10098019900230022FBF770
:1050080019FA431E984131E70000F03F4715F73F72
:1050180044DF5DF80BAE543E0000D03F5555555562
:105028005555D53F0000E03FFE822B650000F0BFDC
:10503800FFFF8F40000070BFC04B00222B420AD1F7
:10504800009801990022BE4BFCF75AF935220090CE
:105058000191019C5242BB4923155B189B182403FC
:10506800B94D0D93B94B220B154300249A4209DD23
:10507800B74B01349A4205DD0D9B1B1900240D9393
:10508800B44BED18E3000F93B34BE2009B18009864
:1050980001991A685B68290006000A920B93FCF7CD
:1050A8009BFB32002B00109011910A980B99FBF78B
:1050B800E9F902000B000020A349FBF71FFD0200DD
:1050C8000B001290139110981199FCF719F9089098
:1050D8000991089A099B80210492059300232F00C7
:1050E80089056D100D4380210493049A059B009255
:1050F8000193002209036D18A1046B180098019907
:1051080014001D00FCF7FCF802000B001098119920
:10511800FCF762FB0A9A0B9B109011912000290062
:10512800FCF75AFB02000B0030003900FCF754FB77
:10513800009A019BFCF7E4F802000B001098119903
:10514800FCF74AFB129A139BFCF7DAF8089A099BBA
:105158000A900B9110001900FCF7D2F806000F0016
:105168007E4A7F4BFCF7CCF87E4A7F4BFBF78AF9E7
:1051780032003B00FCF7C4F87C4A7D4BFBF782F910
:1051880032003B00FCF7BCF87A4A7B4BFBF77AF914
:1051980032003B00FCF7B4F8784A794BFBF772F918
:1051A80032003B00FCF7ACF8764A774BFBF76AF91C
:1051B800320004000D003B0030003900FCF7A0F875
:1051C80002000B0020002900FCF79AF8009A019BC6
:1051D80004000D0008980999FBF754F90A9A0B9BEB
:1051E800FCF78EF822002B00FBF74CF9009A019B84
:1051F8001090119110001900FCF782F80022634BFF
:1052080004000D00FBF73EF9109A119BFBF73AF9E1
:1052180000260F0032000B0000980199FCF770F887
:10522800002200900191594B30003900FCF7D4FA64
:1052380022002B00FCF7D0FA02000B0010981199FD
:10524800FCF7CAFA089A099BFCF75AF832000400DE
:105258000D000A980B993B00FCF752F802000B006E
:1052680020002900FBF70EF904000D0002000B00D6
:1052780000980199FBF706F90026E022444B120634
:1052880030000F00FCF73CF808900991009A019B48
:1052980039003000FCF7A0FA02000B0020002900BA
:1052A800FCF79AFA3B4A3A4BFCF72AF83A4A0400C8
:1052B8000D003A4B39003000FCF722F802000B00D1
:1052C80020002900FBF7DEF80F9A354B9B181A6867
:1052D8005B68FBF7D7F80A900B910D98FCF762FE14
:1052E80004000D00089809990F9A2E4B9B181A680C
:1052F8005B68009201930A9A0B9BFBF7C3F8009A2C
:10530800019BFBF7BFF822002B00FBF7BBF822003C
:105318002B0030000F00FCF75FFA009A019BFCF7A6
:105328005BFA089A099BFCF757FA02000B000A98E7
:105338000B9919E60023044C22E6C0460000F07FD2
:105348000000404301FCFFFF0000F03F8E9803007F
:1053580079B60B000000F0FF007E0008EF4E454ACA
:10536800287ECA3F65DBC9934A86CD3F01411DA906
:105378006074D13F4D268F515555D53FFFAB6FDB3C
:10538800B66DDB3F033333333333E33F000008406C
:1053980009C7EE3FFD033ADCF5015B14E02F3EBE82
:1053A800207E0008107E0008904A914B04980599C9
:1053B800FBF768F83200029003913B0028002100B7
:1053C800FCF70AFA02000B0002980399FBF746F86B
:1053D800002800D00FE60021864A63005B0802918E
:1053E800934225DD844A1B159B188022520394465C
:1053F8001A411419814B6000814D400DC0180541B8
:105408002100A9430B0061462403240B21431424E3
:10541800201A0141029108990022002902DA029912
:105428004942029130003900FCF7D6F906900791FD
:10543800049A059B069807990026FBF723F8002293
:105448003000704B0F00FBF75BFF069A079B089034
:10545800099130003900FCF7BFF902000B000498ED
:105468000599FCF7B9F9684A684BFBF749FF684AA0
:1054780004000D0030003900664BFBF741FF0200C5
:105488000B0020002900FAF7FDFF04000D000200C0
:105498000B0008980999FAF7F5FF089A099B060086
:1054A8000F00FCF799F902000B0020002900FCF717
:1054B80093F93200049005913B0030003900FBF766
:1054C8001FFF04000D00544A544BFBF719FF544AC0
:1054D800544BFCF781F922002B00FBF711FF524ACD
:1054E800524BFAF7CFFF22002B00FBF709FF504A77
:1054F800504BFCF771F922002B00FBF701FF4E4AD5
:105508004E4BFAF7BFFF22002B00FBF7F9FE020013
:105518000B0030003900FCF75FF904000D000200B1
:105528000B0030003900FBF7EBFE80230690079153
:10553800002220002900DB05FCF74EF902000B00D1
:1055480006980799FBF7DAFA049A059B04000D0000
:1055580030003900FBF7D4FE049A059BFAF792FF56
:1055680002000B0020002900FCF736F932003B004E
:10557800FCF732F902000B0000203149FCF72CF946
:10558800029B1B055B181A15002A25DC029A00F0FD
:1055980055F9009A019BFFF733FC2A4A4B005B0838
:1055A800934200DC17E7284BCB18034308D0009838
:1055B800019900230022FAF73DFF431E984162E457
:1055C80032003B00FCF708F9049A059BFAF750FFF4
:1055D800002800D1FFE6EAE71900DAE70023184CB3
:1055E800FFF7F1FB00230024FFF7EDFBFE822B659C
:1055F8004715973C0000E03F02FCFFFF01FCFFFF5E
:10560800FFFF0F00432EE63FEF39FAFE422EE63F3A
:10561800396CA80C615C20BED0A4BE726937663EA6
:10562800F16BD2C541BDBB3E2CDE25AF6A56113F9A
:1056380093BDBE166CC1663F3E5555555555C53F81
:105648000000F03FFFCB904000346F3FF0B50B00F7
:105658000C00564905000200080085B02040884229
:105668000FD128002100FBF74BFE02000B00280099
:105678002100FAF707FF05000C002800210005B0FB
:10568800F0BD002C10DC610049082943F5D0002149
:105698008C4200D180E028002100FCF79DF8020030
:1056A8000B00FBF72BFAE6E7211575D040481B03E2
:1056B8000C1880201B0B40030343C90703D4D10FE8
:1056C8005B005B1852006110002403915B00D10F4E
:1056D8005B188021162520005200890346189E4237
:1056E80002DC70189B1B6418D60F5B00013DF31891
:1056F80052004908002DF1D1202680272900019663
:105708003F067E19B446834202DC14D1964212D871
:1057180065466646ED190290002E03DAEE43F60F51
:10572800861902961B1A6245804140421B1A604640
:10573800121A0298C919D60F5B009B19019E5200D4
:10574800013E7F080196002EDBD1134303D04B1C8A
:1057580027D131000134174B6010C0184908E307FE
:1057680002D580231B061943039B0D001C05231833
:105778001C0082E7D30A15385205002BFAD0802482
:10578800640323420AD020241600641AE6404D1E02
:105798008A403343411B89E70020EEE75B00013173
:1057A800EFE7012301319943D5E7C0460000F07FB8
:1057B80001FCFFFF0000E03F70B50D00160004007B
:1057C800FEF7B4FF29000660200070BD37B515004C
:1057D8001C00002810D0802310001B06E118009040
:1057E8000191009A019B28002100FBF789FD2222E4
:1057F800FFF7E2FF03B030BD10001900EFE7802388
:1058080010B500225B05FFF7E1FF10BDE02310B5DE
:105818000022DB05FFF7DAFF10BD4B00590870477F
:10582800024B48004008C018C00F704700001080A5
:10583800002001497047C0460000F87F4B0070B552
:105848005B0D14000A00002B0DD14B005B080343CD
:1058580010D0274B0022FBF753FD264B9C420ADA57
:10586800254A264B19E0264DAB4208D102000B0011
:10587800FAF708FE70BD0A004B005B0D363B214D60
:10588800E318AB420CDD204C204D002901DA1E4CF8
:105898001F4D200029001C4A1C4BFBF731FDE9E78E
:1058A800002B05DD1B4C1B0522401A431100E1E7C4
:1058B8001D00353513DA184ACB0F944208DD12481B
:1058C8001249002B01D0104811490F4A0F4BE4E749
:1058D80009480A49002BC3D007481049C0E70D4CB6
:1058E800363322401B051343190000220C4BD4E722
:1058F80000005043B03CFFFF59F3F8C21F6EA501EA
:10590800FF070000FE0700009C7500883CE4377E16
:105918003CE437FEFFFF0F8050C300001F6EA581D7
:105928000000903CF8B5C046F8BC08BC9E467047DD
:0C593800F8B5C046F8BC08BC9E4670479D
:10594800E00B0008CE0B0008AC0B0008D60B0008D3
:10595800AC0B0008AE0E0008AC0B0008D60B000814
:10596800CE0B0008CE0B0008AE0E0008D60B0008C0
:10597800980B0008980B0008980B0008240F0008E3
:10598800EE130008AC130008AC130008A8130008B5
:10599800B2130008B2130008BE160008A8130008C6
:1059A800B2130008BE160008B2130008A8130008B6
:1059B8005216000852160008521600082817000848
:1059C8004B61706163697461202546202020202086
:1059D800005A61646E79206B6F6E64656E7A6174CB
:1059E8006F72004F64706F7220254F686D20202001
:1059F80020004F70656E20252C20252C20252C207A
:105A0800250A0D0053686F72742070203D20254FC1
:105A1800686D202C6E203D20254F686D0A0D0041D1
:105A2800646320252C20250A0D00282B29202D7C95
:105A38003E7C2D20282D2920416E6F6461206E61E7
:105A4800202B2073766F72636520200A0D58202062
:105A58002020202020202020202044696F646120FD
:105A680020202020202020202020202020200A0D57
:105A7800582020205564203D2025562040202541CF
:105A8800202020202020202020202020202020200E
:105A9800200A0D582020205564203D2025562040FE
:105AA80020254120202020202020202020202020C8
:105AB800202020200A0D58202020506172616D6539
:105AC800747279206D6F64656C7520202020202009
:105AD800202020202020200A0D582020206E203D44
:105AE80020252C204973203D2025412020202020DE
:105AF800202020202020202020200A0D582020208F
:105B0800202020202020202020202020202020208D
:105B1800202020202020202020202020202020009D
:105B2800282B29202D7C3C7C2D20282D2920416ED6
:105B38006F6461206E61202D2073766F726365201B
:105B4800200A0D582020202020202020202020203E
:105B580044696F64612020202020202020202020FC
:105B6800202020200A0D582020205564203D202583
:105B780056204020254120202020202020202020A1
:105B8800202020202020200A0D5820202055642085
:105B98003D2025562040202541202020202020205F
:105BA800202020202020202020200A0D58202020DE
:105BB800506172616D65747279206D6F64656C7582
:105BC800202020202020202020202020200A0D58BE
:105BD8002020206E203D20252C204973203D2025A3
:105BE800412020202020202020202020202020208C
:105BF8000A0D58202020202020202020202020208E
:105C0800202020202020202020202020202020208C
:105C1800202020202000282B29202D7C3E7C2D2090
:105C2800282D2920416E6F6461206E61202B20731E
:105C3800766F72636520200A0D58202020202020CE
:105C480020205E5E2020466F746F64696F64612057
:105C5800202020202020202020200A0D582020202D
:105C680020202020207C7C20202020202020202074
:105C7800202020202020202020202020200A0D580D
:105C88002020204972203D2025412020202020204E
:105C980020202020202020202020202020202020FC
:105CA8000A0D58202020556430203D2025562040DC
:105CB80020254120202020202020202020202020B6
:105CC8002020200A0D58202020556466203D2025DC
:105CD8005620402025412020202020202020202040
:105CE8002020202020200A0D58202020202020209D
:105CF800202020202020202020202020202020209C
:105D080020202020202020202020200D00282B29A2
:105D1800202D7C3C7C2D20282D2920416E6F64612C
:105D2800206E61202D2073766F72636520200A0D26
:105D38005820202020202020205E5E2020466F74DE
:105D48006F64696F6461202020202020202020209B
:105D5800200A0D5820202020202020207C7C202074
:105D6800202020202020202020202020202020202B
:105D7800202020200A0D582020204972203D20256F
:105D880041202020202020202020202020202020EA
:105D9800202020202020200A0D5820202055643063
:105DA800203D20255620402025412020202020204D
:105DB800202020202020202020200A0D58202020CC
:105DC800556466203D20255620402025412020206E
:105DD800202020202020202020202020200A0D58AC
:105DE80020202020202020202020202020202020AB
:105DF800202020202020202020202020202020209B
:105E0800202000282B29202D5F5F3E2D20282D29BA
:105E1800204B206E61202B2073766F7263652020E3
:105E2800202020200A0D5820202020202020205E1D
:105E38005E2020466F746F7472616E736973746F3D
:105E4800722020202020200A0D58202020202020E9
:105E580020207C7C20202020202020202020202082
:105E6800202020202020202020200A0D582020201B
:105E7800496B203D20254120202020202020202063
:105E8800202020202020202020202020200A0D58FB
:105E980020202020202020202020202020202020FA
:105EA80020202020202020202020202020202020EA
:105EB8000A0D5820202020202020202020202020CB
:105EC80020202020202020202020202020202020CA
:105ED8002020200A0D5820202020202020202020AB
:105EE80020202020202020202020202020202020AA
:105EF800202020202020202000282B29202D3C5F36
:105F08005F2D20282D29204B206E61202D207376AF
:105F18006F7263652020202020200A0D5820202041
:105F28002020202020205E5E2020466F746F74722F
:105F3800616E736973746F7220202020200A0D58D7
:105F48002020202020202020207C7C202020202091
:105F58002020202020202020202020202020202039
:105F68000A0D58202020496B203D20254120202063
:105F78002020202020202020202020202020202019
:105F88002020200A0D5820202020202020202020FA
:105F980020202020202020202020202020202020F9
:105FA8002020202020200A0D5820202020202020DA
:105FB80020202020202020202020202020202020D9
:105FC8002020202020202020200A0D5820202020BA
:105FD80020202020202020202020202020202020B9
:105FE80020202020202020202020202020200028C1
:105FF8002B29202D782D20282D29206E657A6E6179
:106008006D6120736F75636173746B61202020204C
:106018000A0D58202020556466203D202556204032
:106028002025412020202020202020202020202042
:106038002020200A0D58202020556466203D202568
:1060480056204020254120202020202020202020CC
:106058002020202020200A0D5820202055643020A0
:106068003D2025562040202541202020202020208A
:106078002020202020202020200A0D5820202055D4
:106088006430203D20255620402025412020202016
:106098002020202020202020202020200A0D5820E9
:1060A8002020556472203D2025562040202541207F
:1060B8002020202020202020202020202020200AEE
:1060C8000D58202020556472203D20255620402060
:1060D8002541202020202020202020202020202092
:1060E8002020202000455352203D20254F686D0A6E
:1060F8000D001B5B303B313B303B33303B34306D64
:106108001B5B303B313B303B33303B34376D1B5BE3
:10611800303B306658585858585858585858585856
:1061280058585858585858585858585858585858E7
:1061380058585858585858585858585858585858D7
:1061480058585858585858580A0D582020205576ED
:106158006F646E6920737472616E6B6120202020F9
:106168002020202020202020202020202020202027
:1061780020202020202020202020202020580A0D08
:106188005820202054657374657220736F7563619D
:106198007374656B2070726F2053544D33324730DF
:1061A80033304A3620202020202020202020202084
:1061B800202020580A0D582020205A61706F6A65E7
:1061C8006E6920746573746572752028646F706FCA
:1061D800727563656E6520686F646E6F7479206F81
:1061E80064706F727529202020580A0D58202020CD
:1061F8002020202020202020202020202020202097
:106208002020202020202020202020202020202086
:10621800202020202020202020202020202020583E
:106228000A0D58202050696E79202038202020201F
:10623800202020202020203720202020202020203F
:106248002034202020202020202020202031202021
:106258002020202020580A0D582020494F20202097
:106268002028504131352920202020202028504145
:106278003133292020202028504130292020202077
:106288002020202850423729202020580A0D582045
:106298002020202020202020207C2020202020209A
:1062A80020202020207C2020202020202020207C2E
:1062B80020202020202020202020207C202020207A
:1062C80020580A0D582020202020202020202D2D65
:1062D8002D2020202020202020202D2D2D20202082
:1062E80020202020207C202020202020202020204A
:1062F800207C2020202020580A0D582020202020F3
:10630800202020207C207C202020202020202020CD
:106318007C207C20202020202020207C2020202061
:10632800202020202020207C2020202020580A0DFA
:10633800582020205231202020207C207C202052F0
:106348002020202020207C207C202020202020208D
:10635800207C20202020202020202020207C20207D
:10636800202020580A0D582020202833394B292076
:106378007C207C2020283437305229207C207C2027
:10638800202020202020207C2020202020202020A9
:106398002020207C2020202020580A0D5820202052
:1063A8002020202020202D2D2D20202020202020BE
:1063B80020202D2D2D20202020202020207C202052
:1063C8002020202020202020207C20202020205831
:1063D8000A0D58202020202020202020207C20204A
:1063E8002020202020202020207C20202020202049
:1063F8002020207C20202020202020202020207CDD
:106408002020202020580A0D58202020202020203D
:10641800202020582D2D2D2D2D2D2D2D2D2D2D5875
:106428002D2D2D2D2D2D2D2D2D582D2D2D4F202061
:10643800204F2D2D2D582020202020580A0D58207F
:106448002020202020202020202020202020202044
:106458002020202020202020202020202020202034
:106468002020202B2020202D20202020202020200C
:1064780020580A0D582020202020202020202020CD
:106488002020202020202020202020202020202004
:1064980020202020202020202020202020202020F4
:1064A80020202020202020580A0D58202020287045
:1064B80029202D20706F6B7261636F766174207371
:1064C80020646F706F727563656E796D6920686F8F
:1064D800646E6F74616D69202020202020580A0D99
:1064E80058202020287629202D20766C6173746E20
:1064F8006920686F646E6F7479206F64706F72754D
:106508002020202020202020202020202020202083
:10651800202020580A0D582020202020202020202C
:106528002020202020202020202020202020202063
:106538002020202020202020202020202020202053
:10654800202020202020202020580A0D5858585854
:1065580058585858585858585858585858585858B3
:1065680058585858585858585858585858585858A3
:106578005858585858585858585858585858585893
:106588000A0D001B5B303B313B303B33303B343032
:106598006D1B5B303B313B303B33303B34376D1B3D
:1065A8005B303B30665858585858585858585858BF
:1065B8005858585858585858585858585858585853
:1065C8005858585858585858585858585858585843
:1065D8005858585858585858580A0D58202020507C
:1065E80072766F746E6920736572697A656E692058
:1065F8002020202020202020202020202020202093
:106608002020202020202020202020202020580A60
:106618000D5820202054657374657220736F75635C
:10662800617374656B2070726F2053544D33324719
:106638003033304A362020202020202020202020DF
:1066480020202020580A0D582020202020202020FB
:106658002020202020202020202020202020202032
:106668002020202020202020202020202020202022
:1066780020202020202020202020580A0D582020CB
:1066880020312E204E656368746520746573746FBD
:10669800766163692073766F726B7920726F7A7096
:1066A8006F6A656E65206120202020202020202030
:1066B800580A0D582020202020207A6D61636B6EC7
:1066C800657465206B6C617665737520286F292069
:1066D80020202020202020202020202020202020B2
:1066E800202020202020580A0D58202020322E203B
:1066F8005A6B726174756A746520746573746F7609
:106708006163692073766F726B7920612020202085
:10671800202020202020202020202020580A0D582A
:106728002020202020207A6D61636B6E65746520BF
:106738006B6C6176657375202873292020202020D2
:106748002020202020202020202020202020202041
:106758002020580A0D58202020332E205A6D6163BE
:106768006B6E657465206B6C617665737520287037
:10677800292070726F20706F6B7261636F76616E23
:106788006920202020202020580A0D582020202869
:1067980070726F20706F757A6974692064656661BC
:1067A800756C747520707265736B6F637465207295
:1067B8006F766E6F75206E61203329202020580A6D
:1067C8000D58202020446562756720646174613A21
:1067D80020202020202020202020202020202020B1
:1067E80020202020202020202020202020202020A1
:1067F80020202020580A0D5820202020202020204A
:106808002020202020202020202020202020202080
:106818002020202020202020202020202020202070
:1068280020202020202020202020580A0D58202019
:106838002020202020202020202020202020202050
:106848002020202020202020202020202020202040
:106858002020202020202020202020202020202030
:10686800580A0D58202020202020202020202020D9
:106878002020202020202020202020202020202010
:106888002020202020202020202020202020202000
:10689800202020202020580A0D58202020202020A9
:1068A80020202020202020202020202020202020E0
:1068B80020202020202020202020202020202020D0
:1068C800202020202020202020202020580A0D5879
:1068D80020202020202020202020202020202020B0
:1068E80020202020202020202020202020202020A0
:1068F8002020202020202020202020202020202090
:106908002020580A0D582020202020202020202038
:10691800202020202020202020202020202020206F
:10692800202020202020202020202020202020205F
:106938002020202020202020580A0D582020202008
:10694800202020202020202020202020202020203F
:10695800202020202020202020202020202020202F
:106968002020202020202020202020202020580AFD
:106978000D582020202020202020202020202020EA
:1069880020202020202020202020202020202020FF
:1069980020202020202020202020202020202020EF
:1069A80020202020580A0D58202020202020202098
:1069B80020202020202020202020202020202020CF
:1069C80020202020202020202020202020202020BF
:1069D80020202020202020202020580A0D585858F8
:1069E800585858585858585858585858585858581F
:1069F800585858585858585858585858585858580F
:106A080058585858585858585858585858585858FE
:106A1800580A0D001B5B303B313B303B33303B3475
:106A2800306D1B5B303B313B303B33303B34376D93
:106A38001B5B303B30665858585858585858585867
:106A480058585858585858585858585858585858BE
:106A580058585858585858585858585858585858AE
:106A6800585858585858585858580A0D58202020DF
:106A7800486C61766E69206D656E75202020202037
:106A880020202020202020202020202020202020FE
:106A980020202020202020202020202020202058B6
:106AA8000A0D5820202054657374657220736F7521
:106AB80063617374656B2070726F2053544D333269
:106AC800473033304A362020202020202020202024
:106AD8002020202020580A0D582020202020202067
:106AE800202020202020202020202020202020209E
:106AF800202020202020202020202020202020208E
:106B08002020202020202020202020580A0D582036
:106B18002020287229202D20746573746F76616E89
:106B280069206F64706F727520202020202020203B
:106B3800202020202020202020202020202020204D
:106B480020580A0D58202020286329202D207465FC
:106B580073746F76616E69206B6F6E64656E7A61AF
:106B6800746F7275202020202020202020202020D3
:106B780020202020202020580A0D5820202028647A
:106B880029202D20746573746F76616E6920706F8B
:106B98006C6F766F64696375202020202020202088
:106BA80020202020202020202020202020580A0DCE
:106BB8005820202020202020202020202020202095
:106BC80020202020202020202020202020202020BD
:106BD80020202020202020202020202020202020AD
:106BE800202020580A0D5820202020202020202056
:106BF800202020202020202020202020202020208D
:106C0800202020202020202020202020202020207C
:106C1800202020202020202020580A0D5820202025
:106C2800202020202020202020202020202020205C
:106C3800202020202020202020202020202020204C
:106C48002020202020202020202020202020205804
:106C58000A0D58202020202020202020202020201D
:106C6800202020202020202020202020202020201C
:106C7800202020202020202020202020202020200C
:106C88002020202020580A0D5820202020202020B5
:106C980020202020202020202020202020202020EC
:106CA80020202020202020202020202020202020DC
:106CB8002020202020202020202020580A0D582085
:106CC80020202020202020202020202020202020BC
:106CD80020202020202020202020202020202020AC
:106CE800202020202020202020202020202020209C
:106CF80020580A0D58202020202020202020202045
:106D0800202020202020202020202020202020207B
:106D1800202020202020202020202020202020206B
:106D280020202020202020580A0D58202020202014
:106D3800202020202020202020202020202020204B
:106D4800202020202020202020202020202020203B
:106D580020202020202020202020202020580A0D1C
:106D680058202020202020202020202020202020E3
:106D7800202020202020202020202020202020200B
:106D880020202020202020202020202020202020FB
:106D9800202020580A0D58202020202020202020A4
:106DA80020202020202020202020202020202020DB
:106DB80020202020202020202020202020202020CB
:106DC800202020202020202020580A0D5820202074
:106DD80020202020202020202020202020202020AB
:106DE800202020202020202020202020202020209B
:106DF8002020202020202020202020202020205853
:106E08000A0D58202020287529202D207A706574B5
:106E1800206E612075766F646E6920737472616E7E
:106E28006B752020202020202020202020202020BA
:106E38002020202020580A0D582020202020202003
:106E4800202020202020202020202020202020203A
:106E5800202020202020202020202020202020202A
:106E68002020202020202020202020580A0D58589B
:106E7800585858585858585858585858585858588A
:106E8800585858585858585858585858585858587A
:106E9800585858585858585858585858585858586A
:106EA80058580A0D001B5B303B313B303B33303BBD
:106EB80034306D1B5B303B313B303B33303B343738
:106EC8006D1B5B303B3066585858585858585858BE
:106ED800585858585858585858585858585858582A
:106EE800585858585858585858585858585858581A
:106EF80058585858585858585858580A0D58202013
:106F080020546573746F76616E69206F64706F7258
:106F18007520202020202020202020202020202014
:106F28002020202020202020202020202020202059
:106F3800580A0D5820202054657374657220736FA9
:106F48007563617374656B2070726F2053544D3391
:106F580032473033304A362020202020202020207D
:106F6800202020202020580A0D58202020202020D2
:106F78002020202020202020202020202020202009
:106F880020202020202020202020202020202020F9
:106F9800202020202020202020202020580A0D58A2
:106FA80020202020202020202020202020202020D9
:106FB80020202020202020202020202020202020C9
:106FC80020202020202020202020202020202020B9
:106FD8002020580A0D582020202020202020202062
:106FE8002020202020202020202020202020202099
:106FF8002020202020202020202020202020202089
:107008002020202020202020580A0D582020202031
:107018002020202020202020202020202020202068
:107028002020202020202020202020202020202058
:107038002020202020202020202020202020580A26
:107048000D58202020202020202020202020202013
:107058002020202020202020202020202020202028
:107068002020202020202020202020202020202018
:1070780020202020580A0D582020202020202020C1
:1070880020202020202020202020202020202020F8
:1070980020202020202020202020202020202020E8
:1070A80020202020202020202020580A0D58202091
:1070B80020202D20202020202020202020202020BB
:1070C80020202020202020202020202020202020B8
:1070D80020202020202020202020202020202020A8
:1070E800580A0D5820202020202020202020202051
:1070F8002020202020202020202020202020202088
:107108002020202020202020202020202020202077
:10711800202020202020580A0D5820202020202020
:107128002020202020202020202020202020202057
:107138002020202020202020202020202020202047
:10714800202020202020202020202020580A0D58F0
:107158002020202020202020202020202020202027
:107168002020202020202020202020202020202017
:107178002020202020202020202020202020202007
:107188002020580A0D5820202020202020202020B0
:1071980020202020202020202020202020202020E7
:1071A80020202020202020202020202020202020D7
:1071B8002020202020202020580A0D582020202080
:1071C80020202020202020202020202020202020B7
:1071D80020202020202020202020202020202020A7
:1071E8002020202020202020202020202020580A75
:1071F8000D58202020202020202020202020202062
:107208002020202020202020202020202020202076
:107218002020202020202020202020202020202066
:1072280020202020580A0D5820202020202020200F
:107238002020202020202020202020202020202046
:107248002020202020202020202020202020202036
:1072580020202020202020202020580A0D582020DF
:107268002020287029202D206E6176726174206498
:107278006F20686C61766E69686F206D656E752029
:1072880020202020202020202020202020202020F6
:10729800580A0D582020202020202020202020209F
:1072A80020202020202020202020202020202020D6
:1072B80020202020202020202020202020202020C6
:1072C800202020202020580A0D582020202020206F
:1072D80020202020202020202020202020202020A6
:1072E8002020202020202020202020202020202096
:1072F800202020202020202020202020580A0D583F
:1073080058585858585858585858585858585858F5
:1073180058585858585858585858585858585858E5
:1073280058585858585858585858585858585858D5
:107338005858580A0D001B5B31303B3566001B5B03
:10734800303B313B303B33303B34306D1B5B303BA3
:10735800313B303B33303B34376D1B5B303B306661
:107368005858585858585858585858585858585895
:107378005858585858585858585858585858585885
:107388005858585858585858585858585858585875
:10739800585858580A0D58202020546573746F7631
:1073A800616E69206B6F6E64656E7A61746F727559
:1073B80020202020202020202020202020202020C5
:1073C800202020202020202020580A0D582020206E
:1073D80054657374657220736F7563617374656B3C
:1073E8002070726F2053544D3332473033304A3651
:1073F800202020202020202020202020202020584D
:107408000A0D58202020507269206D6572656E69DA
:10741800206B617061636974206E6164203832305A
:10742800206E46206A6520646F62726520202020E5
:107438002020202020580A0D582020206B617061E0
:107448006369747520707269706F6A697420762038
:10745800686C61766E696D206D656E75206120615E
:107468007A2070616B202020202020580A0D582097
:107478002020746573746F7661742020202020208A
:1074880020202020202020202020202020202020F4
:1074980020202020202020202020202020202020E4
:1074A80020580A0D5820202020202020202020208D
:1074B80020202020202020202020202020202020C4
:1074C80020202020202020202020202020202020B4
:1074D80020202020202020580A0D5820202020205D
:1074E8002020202020202020202020202020202094
:1074F8002020202020202020202020202020202084
:1075080020202020202020202020202020580A0D64
:10751800582020202020202020202020202020202B
:107528002020202020202020202020202020202053
:107538002020202020202020202020202020202043
:10754800202020580A0D58202020202D20202020DF
:107558002020202020202020202020202020202023
:107568002020202020202020202020202020202013
:10757800202020202020202020580A0D58202020BC
:1075880020202020202020202020202020202020F3
:1075980020202020202020202020202020202020E3
:1075A800202020202020202020202020202020589B
:1075B8000A0D5820202020202020202020202020B4
:1075C80020202020202020202020202020202020B3
:1075D80020202020202020202020202020202020A3
:1075E8002020202020580A0D58202020202020204C
:1075F8002020202020202020202020202020202083
:107608002020202020202020202020202020202072
:107618002020202020202020202020580A0D58201B
:107628002020202020202020202020202020202052
:107638002020202020202020202020202020202042
:107648002020202020202020202020202020202032
:1076580020580A0D582020202020202020202020DB
:107668002020202020202020202020202020202012
:107678002020202020202020202020202020202002
:1076880020202020202020580A0D582020202020AB
:1076980020202020202020202020202020202020E2
:1076A80020202020202020202020202020202020D2
:1076B80020202020202020202020202020580A0DB3
:1076C800582020202020202020202020202020207A
:1076D80020202020202020202020202020202020A2
:1076E8002020202020202020202020202020202092
:1076F800202020580A0D5820202020287029202DCD
:10770800206E617672617420646F20686C61766E99
:1077180069686F206D656E7520202020202020204C
:10772800202020202020202020580A0D582020200A
:107738002020202020202020202020202020202041
:107748002020202020202020202020202020202031
:1077580020202020202020202020202020202058E9
:107768000A0D582020202020202020202020202002
:107778002020202020202020202020202020202001
:1077880020202020202020202020202020202020F1
:107798002020202020580A0D585858585858585812
:1077A8005858585858585858585858585858585851
:1077B8005858585858585858585858585858585841
:1077C8005858585858585858585858580A0D001B5F
:1077D8005B303B313B303B33303B34306D1B5B30EF
:1077E8003B313B303B33303B34376D1B5B303B30F8
:1077F80066585858585858585858585858585858F3
:1078080058585858585858585858585858585858F0
:1078180058585858585858585858585858585858E0
:1078280058585858580A0D58202020546573746FBA
:1078380076616E6920706F6C6F766F64696375200E
:107848002020202020202020202020202020202030
:1078580020202020202020202020580A0D582020D9
:107868002054657374657220736F756361737465F2
:107878006B2070726F2053544D3332473033304A87
:1078880036202020202020202020202020202020DA
:10789800580A0D5820202020202020202020202099
:1078A80020202020202020202020202020202020D0
:1078B80020202020202020202020202020202020C0
:1078C800202020202020580A0D5820202020202069
:1078D80020202020202020202020202020202020A0
:1078E8002020202020202020202020202020202090
:1078F800202020202020202020202020580A0D5839
:10790800202020202020202020202020202020206F
:10791800202020202020202020202020202020205F
:10792800202020202020202020202020202020204F
:107938002020580A0D5820202020202020202020F8
:10794800202020202020202020202020202020202F
:10795800202020202020202020202020202020201F
:107968002020202020202020580A0D5820202020C8
:1079780020202020202020202020202020202020FF
:1079880020202020202020202020202020202020EF
:107998002020202020202020202020202020580ABD
:1079A8000D582020202020202020202020202020AA
:1079B80020202020202020202020202020202020BF
:1079C80020202020202020202020202020202020AF
:1079D80020202020580A0D58202020202D2020204B
:1079E800202020202020202020202020202020208F
:1079F800202020202020202020202020202020207F
:107A080020202020202020202020580A0D58202027
:107A1800202020202020202020202020202020205E
:107A2800202020202020202020202020202020204E
:107A3800202020202020202020202020202020203E
:107A4800580A0D58202020202020202020202020E7
:107A5800202020202020202020202020202020201E
:107A6800202020202020202020202020202020200E
:107A7800202020202020580A0D58202020202020B7
:107A880020202020202020202020202020202020EE
:107A980020202020202020202020202020202020DE
:107AA800202020202020202020202020580A0D5887
:107AB80020202020202020202020202020202020BE
:107AC80020202020202020202020202020202020AE
:107AD800202020202020202020202020202020209E
:107AE8002020580A0D582020202020202020202047
:107AF800202020202020202020202020202020207E
:107B0800202020202020202020202020202020206D
:107B18002020202020202020580A0D582020202016
:107B2800202020202020202020202020202020204D
:107B3800202020202020202020202020202020203D
:107B48002020202020202020202020202020580A0B
:107B58000D582020202020202020202020202020F8
:107B6800202020202020202020202020202020200D
:107B780020202020202020202020202020202020FD
:107B880020202020580A0D58202020202870292045
:107B98002D206E617672617420646F20686C617646
:107BA8006E69686F206D656E75202020202020206A
:107BB80020202020202020202020580A0D58202076
:107BC8002020287529202D20616B746976616365F2
:107BD80020756E697665727A616C6E69686F20745B
:107BE800657374752020202020202020202020204C
:107BF800580A0D5820202020202020202020202036
:107C0800202020202020202020202020202020206C
:107C1800202020202020202020202020202020205C
:107C2800202020202020580A0D58585858585858B5
:107C380058585858585858585858585858585858BC
:107C480058585858585858585858585858585858AC
:107C5800585858585858585858585858580A0D008D
:107C68001B5B324A1B5B303B30665A6164656A7441
:107C7800652063656C6F636973656C6E6520686FFA
:107C8800646E6F747520522076206F686D65636826
:107C98003A200043687962612C207A6164616E79C8
:107CA800207A6E616B206E656E69206369736C6FF4
:107CB8002C207A6B7573746520746F207A6E6F76DA
:107CC800750A0D000A005A6164656A746520636567
:107CD8006C6F636973656C6E6520686F646E6F7432
:107CE800752052312076206F686D6563683A2000F0
:107CF80052203D20256F686D2C205231203D2025D3
:107D08006F686D0A0D0050726F20706F6B7261633F
:107D18006F76616E69207A6D61636B6E657465203C
:107D28006A616B6F756B6F6C6976206B6C617665D9
:107D380073753A20001B5B31323B3566001B5B31A3
:107D4800333B3566001B5B31343B35660071727915
:107D58007A6166706E756D006B4D475450455A597F
:107D68005251000000000000000000000000000068
:107D780000000000000000000000000000000000FB
:107D880000000000010000000200000003000000E5
:107D980004000000060000000700000008000000C2
:107DA80009000000000000000000000000000000C2
:107DB80000000000010000000200000003000000B5
:107DC80004000000010000000200000004000000A0
:107DD80006000000080000000A0000000C00000077
:107DE800100000002000000040000000800000009B
:107DF8000001000000000000000000000000F03F4B
:107E0800000000000000F83F000000000000000033
:107E18000000004003B8E23F00000000000000003E
:087E280006D0CF43EBFD4C3EF8
:047E3000E100000865
:047E3400B900000889
:107E380001010000000000005C9CEA715996BC3DFD
:107E4800E60F0000FA0F0000020000000200000028
:107E58000000000000607D4000000000000BE340CF
:107E68000000000000003E4000000000000041400B
:107E780000000000000039400024F40050000020F9
:107E880000000000000000000000000000000000EA
:107E980000000000000000000000000000000000DA
:107EA80000000000000000000000000000000000CA
:107EB80000000000000000000000000000000000BA
:107EC80000000000000000000000000000000000AA
:107ED800000000000000000000000000000000009A
:04000005080043515B
:00000001FF
